:046FC600010001487D
:106A3700AF50055074D02FF582E4341DF583E599E6
:106A4700F022D3E5309400E52F94002290000FE068
:036A5700640322B3
:0300030002587B25
:0B587B00C0E0C083C082C0D075D00820
:10588600852E82852D83E493FF201404C4540FFFD4
:10589600430FF08F80C284D28500C2870000D28772
:1058A600007580FF7580FEC284C28500C287000035
:1058B600D287007580FF30140CC214052EE52E70B9
:0958C60006052D8002D214D2A8BF
:0958CF00D0D0D082D083D0E032A9
:03000B000219696E
:10196900C0E0C0F0C083C082C0D075D008758CD8E3
:10197900758A92D28C12422812637AE531D3940087
:1019890040171531E53164056009E531640F6003DD
:10199900021B7B126C7C021B7B753114E54ED394C0
:1019A900004002154EE54FD394004002154FE53A29
:1019B900D394004002153AE54BD394004002154BED
:1019C900154CE54C123A5E1B6D001B42011B1A02B5
:1019D9001AF2031A6F041A56051A3D061A24071A31
:1019E9000B0819F20900001B78D3E52C9400E52BAC
:1019F90094005003021B7BE52C152C704D152B020E
:101A09001B7BD3E5379400E53694005003021B7B1A
:101A1900E537153770021536021B7BD3E54894006C
:101A2900E54794005003021B7BE5481548700215F1
:101A390047021B7BD3E54A9400E549940050030211
:101A49001B7BE54A154A70021549021B7BD3E52A1F
:101A59009400E52994005003021B7BE52A152A709E
:101A6900021529021B7B7884E6FF7003021B7BEFBA
:101A7900B40105900524801BEFB40210126A494095
:101A89002FE53015307002152F021B7BEFB4030CC4
:101A9900900526E0F52FA3E0F5308028EFB4041275
:101AA900126A49400BE53015307002152F021B7B75
:101AB9008012EF64057003021B7BEFB4060C752FCF
:101AC90002753058788406021B7BEF6407600302B5
:101AD9001B7B126A49400BE53015307002152F0245
:101AE9001B7B78847600021B7BD3E5399400E538AB
:101AF90094004008E539153970021538D3E53C944E
:101B090000E53B9400406BE53C153C7002153B80B9
:101B190061D3E5579400E55694004008E5571557F9
:101B290070021556D3E5559400E55494004043E5F9
:101B3900551555700215548039D3E5359400E534AF
:101B490094004008E535153570021534301523D356
:101B5900E5339400E53294004018E53315337012EB
:101B69001532800EE551D39400400415518000755B
:0D1B79004C0AD0D0D082D083D0F0D0E03222
:03001300023EF3B7
:0D3EF300C0E0C0F0C083C082C0D075D01008
:103F0000E545C394504003023FB7202403023FB766
:103F1000300C03023FB7E5A0540FF5587D077F0131
:103F2000124EEA5067202364E545700DE558B40C45
:103F300008201105D211023FB720034A2011471271
:103F40003FC250047F0180027F0F126F4990000F23
:103F5000E0FF64016012EFB40302800C90000FE0F8
:103F6000B40209123FC250047F80801290000FE01B
:103F7000B4020E7D037F07124EEA40057FA01200B7
:103F800016754202D20390053CE0F53A7D087F05A4
:103F9000124EEA502290002BE0B55807202304D29D
:103FA000268014053EE53EAE3D7002053D14F582C7
:073FB0008E83E558F0054582
:103FB700D0D0D082D083D0F0D0E0327D037F0712FB
:033FC7004EEA229D
:0300230002645321
:10645300C0E0C083C082C0D075D018309819C298EC
:10646300E599B40A08126A37755000800AE550C3EB
:1064730094905003126A37309902C299D0D0D082D7
:05648300D083D0E032DF
:03003B0002493047
:0D493000C0E0C0F0C083C082C0D075D018B8
:10493D00C2CEE546C3941040030249C830257C2001
:10494D000C79AFA07804EF08800123D8FDF55953F9
:10495D00590F7D077F02124EEA5035202332E5466E
:10496D00700CE559B40C07201304D213804D2004AC
:10497D001920131690000FE0B4020F7F0A126F4931
:10498D007F80120016754202D20490053CE0F53A84
:10499D007D087F05124EEA502290002BE0B5590795
:1049AD00202304D22880140540E540AE3F70020557
:0B49BD003F14F5828E83E559F005469B
:0B49C800D0D0D082D083D0F0D0E032FD
:104B9500E4F55AF55B755C1E755DFF855B82855A8C
:104BA50083E0F55E635EFFE55EF0E0655E6003123F
:104BB5006FCA635EFF855B82855A83E55EF0E065BB
:104BC5005E6003126FCA055BE55B7002055AE55D21
:104BD500155D7002155CD3E55D9400E55C940050AD
:104BE500BA75985A758921758845758DE7758780D9
:104BF500758CD8758AEF75C90275C808753D1E751F
:104C05003E60753F1E7540B075B701D2A9D2E8D296
:0F4C1500AA75C64C75EEFF75FEFFD2AF1267820F
:014C2400226D
:026FCA0080FE47
:106A1400202F0F90053AE0F54EE54ED39400401236
:106A240080F7302F0D90053AE0F54FE54FD39400F1
:036A340050F922F4
:1069CC0030310AD215900024E04420800DC2157F8E
:1069DC0008126F8A900024E054DFF0FD7F247E00C3
:0469EC0012641D22F2
:102ECA008F6AE56A640170292030047F01805620E8
:102EDA003003022FC5122FD64003022FC5122FDE50
:102EEA00500C122FC6301503022FC5022FBB022F1A
:102EFA007BE56A640270202030047F02802720303C
:102F0A0003022FC5122FE64003022FC5126A53701F
:102F1A0003022FC5022F95E56A64036003022FC5D9
:102F2A002030057F03026F8A303024122FD6501FBB
:102F3A00122FE6501A126A536015122FDE500B7FB9
:102F4A000B122FEE201574022FBB7F03022FC23003
:102F5A003023122FFC501E7D017F02124EEA4015CB
:102F6A007D017F07124EEA5008122FC620154C80A9
:102F7A00407F018043303017122FFC40127D017FC1
:102F8A0002124EEA5009126A5360047F0280293005
:102F9A0030297D017F01124EEA5020126A53701BBC
:102FAA007D017F07124EEA500D7F09122FEE201580
:102FBA000AD2310269CC7F01126F9D227F09126FFA
:102FCA009D900536E0F532A3E0F533227D017F01BD
:102FDA00124EEA227D017F07124EEA227D017F020C
:102FEA00124EEA22126F9D900536E0F532A3E0F503
:0A2FFA0033227D017F01124EEA220E
:104C2500C2957FFF126F8A124B957F071263B150B1
:104C35000512003E8003126138D28C7F081263B1E1
:104C450050051242E880FEC22B1269129000D1E095
:104C5500FF7C117D00125C6C125DDF90000FE0B4EB
:104C65000105122831801090000FE0FF64026004F6
:104C7500EFB40303123265123D32301E11E5427066
:104C85000DE52754A060077FA0126F49C21E7D075E
:104C95007F05124EEA4002C200E552C3940A50BB9A
:104CA5003015B8E533453270B2C2311269CC80ABEC
:104A6C00EF253EFFEE353DCF2401FDE43FFC22AFA8
:104A7C005A7E00EF2403FDEE33FC22E53E255AF569
:104A8C0082E4353DF58322E540255AF582E4353F35
:104A9C00F58322E56F256DF582E4356EF583E0FF35
:104AAC00E56F256DF582E4356EF58322E55A240217
:104ABC00FFE433FE22E56C2401FFE433FEC3E56D15
:104ACC009FEE6480F874809822EF2540FFEE353F0E
:104ADC0022C2017FF47E01126CEEE56C25E0F56CD0
:104AEC00756D0122E55C2EF582E4355BF583E0FD06
:084AFC0022753D1E753E60228B
:106CEE00EF1FAA0670011ED39400EA9400400BE435
:0A6CFE00FDEDC394C850E90D80F7C6
:016D08002268
:105306008F5BE55BB401197D017F06124EEA500CF6
:105316009000B1E0FF7C0D7D00125C6C7884062263
:10532600E55BB4021312537850439000B2E0FF7C61
:105336000D7D20125C6C8035E55BB4041612537843
:10534600500C9000B4E0FF7C0D7D60125C6C78849C
:10535600760622E55BB403197D027F06124EEA50FB
:105366000C9000B3E0FF7C0D7D40125C6C78847677
:0A53760001227D027F06124EEA229A
:104EEA00BF0107900020E0FE8048BF020790002122
:104EFA00E0FE803EBF0307900022E0FE8034BF043C
:104F0A0007900023E0FE802ABF0507900024E0FEF8
:104F1A008020BF0607900025E0FE8016BF07079095
:104F2A000026E0FE800CBF0807900027E0FE800202
:104F3A00E4FEBD0103EE1322BD0204EEA2E122BD8E
:104F4A000304EEA2E222BD0404EEA2E322BD05049C
:104F5A00EEA2E422BD0604EEA2E522BD0704EEA2FB
:074F6A00E622BD0802EE3350
:014F7100221D
:101D8700124AFD900100E0F55A124A87E0123A5EC6
:101D97001DB6011DEB021E20031E55041E8A051EDB
:101DA700BF061EF4071F24081F500900001F7A12E0
:101DB7004A87A3E0B40A15E55A124ABAE545B507BA
:101DC7000BE4B506077D017F01021F38124A7BE548
:101DD700456D7001EC6003021F7A124A6CC2297FBD
:101DE70001021F4D124A87A3E0B40A15E55A124AA9
:101DF700BAE545B5070BE4B506077D017F02021F6B
:101E070038124A7BE5456D7001EC6003021F7A12B8
:101E17004A6CC2297F02021F4D124A87A3E0B40A07
:101E270015E55A124ABAE545B5070BE4B506077D2D
:101E3700017F03021F38124A7BE5456D7001EC6094
:101E470003021F7A124A6CC2297F03021F4D124AEE
:101E570087A3E0B40A15E55A124ABAE545B5070B58
:101E6700E4B506077D017F04021F38124A7BE5456A
:101E77006D7001EC6003021F7A124A6CC2297F045D
:101E8700021F4D124A87A3E0B40A15E55A124ABA4F
:101E9700E545B5070BE4B506077D017F05021F3849
:101EA700124A7BE5456D7001EC6003021F7A124A06
:101EB7006CC2297F05021F4D124A87A3E0B40A1599
:101EC700E55A124ABAE545B5070BE4B506077D01A1
:101ED7007F06021F38124A7BE5456D7001EC6003EF
:101EE700021F7A124A6CC2297F06021F4D124A87C7
:101EF700A3E0B40A14E55A124ABAE545B5070AE45D
:101F0700B506067D017F078028124A7BE5456D707F
:101F170001EC705F124A6CC2297F078029124A8739
:101F2700A3E0B40A0F124A87A3A3E070077D017FDD
:101F370008024E5F124A7BE5456D7001EC70341262
:101F47004A6CC2297F08020FFB124A87A3A3E070DD
:101F570022124A87A3E024F96008147016E4FF02EE
:101F67005FFF7FF47E01126CEE7D5E7F0212675881
:031F77001242E82B
:011F7A002244
:101B8600753F1E7540B0900108E0F55A124A93E081
:101B9600123A5E1BB8011BF0021C28031C60041CD1
:101BA60098051CD0061D08071D3B081D700900007E
:101BB6001D86124A93A3E0B40A13124AB8E546B545
:101BC600070BE4B506077D017F01021D53AF5A12CC
:101BD6004A7DE5466D7001EC6003021D86124AD50A
:101BE600124A73D2297F01021D6D124A93A3E0B4F3
:101BF6000A13124AB8E546B5070BE4B506077D0198
:101C06007F02021D53AF5A124A7DE5466D7001EC04
:101C16006003021D86124AD5124A73D2297F020238
:101C26001D6D124A93A3E0B40A13124AB8E546B5ED
:101C3600070BE4B506077D017F03021D53AF5A1259
:101C46004A7DE5466D7001EC6003021D86124AD599
:101C5600124A73D2297F03021D6D124A93A3E0B480
:101C66000A13124AB8E546B5070BE4B506077D0127
:101C76007F04021D53AF5A124A7DE5466D7001EC92
:101C86006003021D86124AD5124A73D2297F0402C6
:101C96001D6D124A93A3E0B40A13124AB8E546B57D
:101CA600070BE4B506077D017F05021D53AF5A12E7
:101CB6004A7DE5466D7001EC6003021D86124AD529
:101CC600124A73D2297F05021D6D124A93A3E0B40E
:101CD6000A13124AB8E546B5070BE4B506077D01B7
:101CE6007F06021D53AF5A124A7DE5466D7001EC20
:101CF6006003021D86124AD5124A73D2297F060254
:101D06001D6D124A93A3E0B40A12124AB8E546B50D
:101D1600070AE4B506067D017F078031AF5A124AED
:101D26007DE5466D7001EC7057124AD5124A73D2A2
:101D3600297F078032124A93A3E0B40A13124AB8E5
:101D4600E546B5070BE4B506077D017F08024E5F41
:101D5600AF5A124A7DE5466D7001EC7023124AD5E2
:101D6600124A73D2297F08020FFB124A93A3A3E0FB
:101D7600700E124A93A3E024F870057F01125FFFEC
:011D8600223A
:0447E3008C5B8D5C02
:1047E700055CE55C7002055B14F5828C83E0F9706B
:1047F7000302488AEF7005124AFD8009BF0106755A
:104807003F1E7540B0302946EF7007E965456002E5
:10481700C322BF0107E965466002C322E4FEEEC377
:10482700995029EF700F124AF0E53E2E124A8BE09D
:104837006D6002C322EF6401700F124AF0E5402E4B
:10484700124A97E06D6002C3220E80D2D32220293C
:1048570033E4FEEEC3995029EF700F124AF0E53E9C
:104867002E124A8BE06D6016C322EF6401700F129F
:104877004AF0E5402E124A97E06D6002C3220E808F
:04488700D2D322C3A3
:01488B00220A
:060FFB008F5BAB05AA04A8
:101001007D027F07124EEA5011E55BB4050C8B821D
:101011008A83E0640570030212687D017F07124E26
:10102100EA5011E55BB4050C8B828A83E06406709B
:1010310003021268C22AEB24FFF582EA34FFF5832A
:10104100E0F55D8B828A83E0FFF55EA3E0F9F55F51
:10105100EF123A5E107101107802107F03108604BE
:10106100108D05109406109B0710A208000010A710
:10107100755C01D22A802F755C02D22A8028755CAA
:1010810004D22A8021755C08D22A801A755C10D29C
:101091002A8013755C20D22A800C755C40D22A808C
:1010A10005755C80D22AE924FE700302116924F8D7
:1010B100605C2409600302117BE55BB401059000CB
:1010C100208045E55BB40205900021803BE55BB4DF
:1010D10003059000228031E55BB404059000238074
:1010E10027E55BB40505900024801DE55BB406058A
:1010F1009000258013E55BB407059000268009E583
:101101005B64087077900027E0455CF0806EE55BDA
:10111100B401059000208045E55BB40205900021F3
:10112100803BE55BB403059000228031E55BB404AC
:10113100059000238027E55BB40505900024801D00
:10114100E55BB406059000258013E55BB4070590C7
:1011510000268009E55B64087022900027E0FFE526
:101161005CF4FEEF5EF08014E55BB4050D8B828AC2
:1011710083E0FFD22F122992C22AC22A202A030217
:101181001268E55BB40109900020E0FD7F208060DA
:10119100E55BB40209900021E0FD7F218052E55B0F
:1011A100B40309900022E0FD7F228044E55BB40492
:1011B10009900023E0FD7F238036E55BB4050990AB
:1011C1000024E0FD7F248028E55BB406099000251A
:1011D100E0FD7F25801AE55BB40709900026E0FD5C
:1011E1007F26800CE55BB4080C900027E0FD7F278B
:1011F1007E0012641D126DE8D2AF2029047F0180A8
:10120100027F02126F9DA229922F126A14AD5DE432
:10121100FF126758AD5EE4FF126758E55FB4010441
:101221007D388007E55FB40A077D367F061267586F
:10123100E55BB405031265B57D077F05124EEA50E3
:101241000A200007C2307F03122ECA7D017F0112DE
:101251004EEA4005C230122ECA7D017F02124EEACB
:071261004005C230122ECA45
:011268002263
:024E5F008F5B67
:104E6100ED24FF922F126A14E55B123A5E4E8A011D
:104E71004E8F024E94034E99044E9E054EA3064E4C
:104E8100A8074EAD0800004EB3900020802190008D
:104E910021801C9000228017900023801290002412
:104EA100800D90002580089000268003900027E067
:104EB100F55CE55C6024755E01E4F55DE55C30E080
:104EC10007AD5EE4FF126758E55CC313F55C055E50
:104ED100055DE55DC3940840E3227D187F021267FA
:084EE100587D537F021267584F
:014EE90022A6
:1063B100C2AFD284C285BF070BC28600E580A2E2CC
:1063C100922A8019BF080BC28600E580A2E3922AB7
:1063D100800BBF0508C28600E58013922AD286D2BF
:0563E10085D2AFA22AE5
:0163E6002294
:1045CE00C229D22DE4FF125A997D2E7F031267580D
:1045DE007D607F021267587F03126F8A3024FD20A0
:1045EE0024FDE5456407703B7E017F50124AFD8F26
:1045FE00828E837407F07D01E53E2D124A8BE58293
:10460E0024FFF582E58334FFF583E0F9EF2DF58283
:10461E00E43EF583E9F00DBD08DED2297F647E000D
:10462E00126CEE7F081263B15043302995D22DE4FF
:10463E00FF125A997D607F021267587D327F0612F3
:10464E0067587D1E7F05126758C22DE4FF125A99D6
:10465E007C017D507B087F507E011256957F08129B
:10466E0063B150097F327E00126CEE80F07F647E63
:04467E0000126CEECC
:014682002215
:02562C008F5A93
:10562E00900138E0F55BE55A7020E55B124ABAE569
:10563E00456F7001EE704F7460255BF582E4341E89
:10564E00AF82F55D8F5E7F408024E55A640170362F
:10565E00E55B124ABAE5466F7001EE702974B0250B
:10566E005BF582E4341EAF82F55D8F5E7F10120013
:10567E0016855E82855D83E0FFA3E0FD126E368F98
:06568E005CE4FD124F7206
:0156940022F3
:024F72008D6B45
:104F740075F020EF900280123A52AF8285836E8FD3
:104F84006FE0F56CD394004060E56C9410505AE5E2
:104F94006B7014124ADF124AC1504E124A9F124FCC
:104FA400F3056D056D80EFE56B64017019124ADD40
:104FB400124AC15034124A9F124FF33024028029FE
:104FC400056D056D80EAE56B6402701D124ADD1201
:104FD4004AC15015124A9FA3E0FD1265E53024032F
:0E4FE400024D44056D056D80E67F50126F4949
:084FF20022A3E0FD1265E52297
:100D2E00855C82855B83A3A3E0FF855C82855B8304
:100D3E00A3222430F58274003EF583EDF0AF62EF0E
:100D4E003395E0FEE55F2FF582E55E3EF58322E505
:100D5E00822406F582E43583F583E0FF126E11AD31
:100D6E0007AF63EF3395E0FEEF22A3A3E0FFE55C50
:100D7E002404F582E4355BF583E022E55F2405F576
:100D8E0082E4355EF583E022E55F2405F582E435E5
:100D9E005EF583E0FFE55F2406F582E4355EF583BC
:100DAE00E0228E69F56AAF68EF3395E0FEE5662FB7
:100DBE00F582E5653EF583222455F582E4340AF585
:100DCE0083EFF0E56275F007A422AF60EF3395E094
:100DDE00FEE56175F008900158123A52E5822FF542
:100DEE0082E5833EF58322E5662405F582E43565CA
:100DFE00F583E022E55E75F007A42454F582E43411
:100E0E000AF58322A3A3A3E0FF8D828C83E58224BF
:100E1E0004F582E43583F583E022E55E75F007A4E0
:100E2E002451F582E4340AF5832224E0F582740A13
:100E3E003EF583E5822DF582E5833CF58322E55E62
:100E4E0075F007A42453F582E4340AF58322E55F96
:100E5E002405F582E4355EF583E0FFE55F2406F5B3
:100E6E0082E4355EF583E022E55E75F007A4245238
:100E7E00F582E4340AF58322749F2562F582E43408
:100E8E0000F58322746F2562F582E43400F5832227
:100E9E002450F582E4340AF58322ECFF3395E0FE0C
:100EAE00EF25E0FFEE33FE75F02022E5602405F518
:100EBE0082E4355FF58322D3EF6480948022AB0702
:100ECE00AA068B828A83A3A3A3E0FFEB2404F582F8
:100EDE00E43AF583E0FD228F828E83A3A3A3E02262
:100EEE00855F82855E83A3A322AB5DAD5AAF5CAEF8
:100EFE005B22FFE562FD3395E0FCE55F2DF582E5B3
:100F0E005E3CF5832233CE33CE92E022A2E0CE13A6
:100F1E00CE132275F00AA42DFDE5F03CFCE5662209
:100F2E00E5602405F582E4355FF583E022E5627520
:100F3E00F008900158023A52E55E75F007A4245568
:100F4E00F582E4340AF583E022AB5AAD5DAF5CAEB8
:100F5E005B22EF7C002563FDEC35628D82F58322EA
:100F6E00A3A3E0FFAD5A22540FF5657808AF03AE88
:100F7E0002EF08220564E564AE632275F020123A92
:100F8E0052E0FEA3E0FF22E0FAA3E0FB780CFFAEF6
:100F9E00020822E0FCA3E0FD7804FFAE040822E57F
:100FAE00632561F582E43562F58322E5662DF582CF
:100FBE00E5653CF58322E5662FF582E5653EF58312
:100FCE00222431F5827400222480F58274023EAF11
:100FDE0082222560F560E4355FF55F2285608285AB
:0D0FEE005F83228F828E83A3A3E0640A221A
:02055B008F5AB5
:10055D00C22AE4F542D223D22D125A997D4B7F0245
:10056D001267587D02E4FF1267587D32E4FF12676F
:10057D00587D607F021267587D027F07124EEA5048
:10058D00057F04126F8A900528E0F536A3E0F53754
:10059D007F03126F8AE55A7006A22492298009E51D
:1005AD005AB40104A2259229E53745367005D22AA1
:1005BD00020A223029DFE55A7006A2249229800909
:1005CD00E55AB40104A22592292029EAE55A700BB7
:1005DD00755B1E755C6085455D800EE55AB401093D
:1005ED00755B1E755CB085465DE55DD3940050036B
:1005FD00020A1C855C82855B83E0640B6003020A42
:10060D0017A3E0FFB40A0AE55DB40205D22A020A77
:10061D001CEF6401701E120D38A3E0640A7015E51D
:10062D005D6405700F120D38120D78120A4D1231DE
:10063D0038020A1C120D38E0B40111120D38A3E076
:10064D00B40109120EF7121725020A1C120D38E01B
:10065D006401701E120D38A3E064027015E55D642F
:10066D0005700F120D38120D78120A4D1262260206
:10067D000A1C120D38E06401701D120D38A3E064E0
:10068D00037014E55DB4050F120D38120D78FDAB36
:10069D005A123A84020A1C120D38E0B4011D120DD3
:1006AD0038A3E0B40415E55DD39405400EAB5AAD07
:1006BD005CAC5BAF5D123004020A1C120D38E064B5
:1006CD0001701D120D38A3E064057014E55DB405CD
:1006DD000F120D38120D78FDAB5A125B8B020A1CEE
:1006ED00120D38E06401701D120D38A3E064067020
:1006FD0014E55DB4050F120D38120D78FDAB5A12CD
:10070D004DD2020A1C120D38E0B4011D120D38A392
:10071D00E0B40715E55DD39405400EAB5AAD5CAC66
:10072D005BAF5D124683020A1C120D38E064017046
:10073D001D120D38A3E064087014E55DB4050F12A9
:10074D000D38120D78FDAB5A126260020A1C120DA3
:10075D0038E0B40215120D38A3E0B40A0DE55DB40E
:10076D000308AF5A1263E7020A1C120D38E0B402F7
:10077D0016120D38A3E0B4010EE55DB40E09120E8C
:10078D00F9122D8E020A1C120D38E0B40216120D4C
:10079D0038A3E0B4020EE55DB40709120EF9125349
:1007AD00F9020A1C120D38E0B40215120D38A3E03F
:1007BD00B4090DE55DB40308AF5A1255C0020A1C09
:1007CD00120D38E064027019120D38A3E0B409114E
:1007DD00E55DB4040C120D38120F6E1267FE020A9D
:1007ED001C120D38E064037021120D38A3E0640A69
:1007FD007018E55D64057012120D38120D78FD123A
:10080D006E36AD5A124738020A1C120D38E06403D9
:10081D007029120D38A3E064017020E55DD39405B5
:10082D004019120D38120D78FD126E36855A62ABD5
:10083D005DAD5CAC5B123E13020A1C120D38E06418
:10084D00037021120D38A3E064027018E55D640594
:10085D007012120D38120D78FD126E36AD5A1260EF
:10086D007F020A1C120D38E0B40315120D38A3E0F7
:10087D00B4030DE55DB40308AF5A1260FB020A1C08
:10088D00120D38E0B40318120D38A3E0B40410E5CE
:10089D005DD394034009120F571249D3020A1C125B
:1008AD000D38E0B40315120D38A3E0B4050DE55D68
:1008BD00B40308AF5A126E24020A1C120D38E0B4AC
:1008CD000316120D38A3E0B4060EE55DB40509124A
:1008DD000EF9126938020A1C120D38E06403701902
:1008ED00120D38A3E0B40711E55DB4040C120D38F8
:1008FD00120F6E126C42020A1C120D38E0B4031670
:10090D00120D38A3E0B4080EE55DB40409120EF91A
:10091D0012695D020A1C120D38E064057014E55D64
:10092D00B4040F120D2EA3A3E0FDAB5A121F7B02D0
:10093D000A1C120D38E0B40516120D7CB40B10E52F
:10094D005DD394054009120F57123391020A1C1200
:10095D000D38E064067014E55DB4040F120D2EA37E
:10096D00A3E0FDAB5A12216D020A1C120D38E0B442
:10097D000616120D7CB40B10E55DD39405400912DB
:10098D000F571226A8020A1C120D38E06409701ABE
:10099D00120D38A3E0B40A12E55DB4040D120D3842
:1009AD00A3A3E0FF125E28020A1C120D38E06409B1
:1009BD007018120D38A3E0B40110E55DB4040B12EC
:1009CD000D38120F6E1263438045120D38E0B409D5
:1009DD0017120D38A3E0B4020FE55DD3940440085F
:1009ED00120EF71214D78027120D38E06409701A11
:1009FD00120D38A3E0B40310E55DB4040B120D38ED
:100A0D00120F6E125D9680078000AF5A126C5F2038
:100A1D002A030205A2C21ED22DAF5A125A997D6029
:100A2D007F021267587D327F031267587F03126F62
:0F0A3D008A125E707FFF126F49E47884F6C2233D
:080A4C0022FD126E36AD5A22A4
:081725008E5E8F5F8D608B6109
:10172D00120EE5FFE55F2404120D8DFD1264F08F9E
:10173D006274E22562F562C394005003021926E536
:10174D006294144003021926E5616406701D120DA2
:10175D0089B4010C120DD1120E9E7401F0021922E2
:10176D00120DD1120E9EE4F0021922E561640E6095
:10177D0003021844E55F240C120D8DFFB40A14E525
:10178D005F240D120D8DB40A0A120DD1120E2EE426
:10179D00F08013E55F240D120D8DFD126CB6120D48
:1017AD00D1120E2EEFF0E55F240A120D8DFFB40A53
:1017BD0014E55F240B120D8DB40A0A120DD1120E11
:1017CD007CE4F08013E55F240B120D8DFD126CB6D9
:1017DD00120DD1120E7CEFF0E55F2409120D8DFF75
:1017ED00640A6006EFD39409400A120DD1120E520D
:1017FD00E4F08010E55F2409120D8DFF120DD1125A
:10180D000E52EFF0120D89FFB40B15E55F24061291
:10181D000D8DB40B0B120DD1120E0874FFF0800854
:10182D00121952120E08EFF012192E120DC6120EC9
:10183D009E7401F0021922E561640A706E120DD1D9
:10184D00120E2EE4120DD0120E7CE4F0E55F240989
:10185D00120D8DFF640A6006EFD39409400A120D34
:10186D00D1120E52E4F08010E55F2409120D8DFFA8
:10187D00120DD1120E52EFF0120D89FFB40B15E5BA
:10188D005F2406120D8DB40B0B120DD1120E0874C0
:10189D00FFF08008121952120E08EFF012192E12D5
:1018AD000DC6120E9E7401F0021922E561640970D5
:1018BD0068120DD1120E2EE4120DD0120E7CE41210
:1018CD000DD0120E52E4F0120D89FFB40B15E55F29
:1018DD002406120D8DB40B0B120DD1120E0874FFD0
:1018ED00F08013E55F2406120D8DFD126CB6120DFE
:1018FD00D1120E08EFF0E55F2407120D8DFFE55FA5
:10190D002408120D8DFD126CB6120DD1120DC612DA
:10191D000E9E7401F0D22C8002C22CAF60126F1F8C
:10192D0022E55F2407F582E4355EF583E0FFE55F90
:10193D002408F582E4355EF583E0FD126CB6E562B0
:10194D0075F007A422E55F2406F582E4355EF58384
:0C195D00E0FD126CB6E56275F007A422F4
:103138008F5E8D5FE55ED3941D5003023244E55ED9
:1031480094324003023244D22DAF5F125A997D4621
:103158007F07126758AF5E1235B874E2255EF55ED8
:10316800120E2AE07021120E76E0701B120E4CE04F
:103178007015120E02E0700F120F46700A12325DBF
:103188007D537F0202323A12324CE55E75F007A495
:10319800120E9EE070047D3680027D387F0612672D
:1031A8005812324C120E28E0FFD394014034EF94A9
:1031B80013502F7D097F06126758120E28123254B9
:1031C8007FF47E01126CEE7D0E7F031267587D3509
:1031D8007F061267587D097F06126758120E76120D
:1031E80032547FF47E01126CEE120E4CE0FF600543
:1031F800125B3C800A12325D7D0F7F031267587D97
:10320800277F02126758120E02E0FFF46008126D61
:10321800731235B880077D187F021267587D377F93
:1032280004126758120F46FF126D731235B87D05E8
:103238007F06126758C22DAF5F025A99C22CAF5F42
:10324800126F1F227FF47E01126CEE22E0FF126DD6
:0D325800731235B8227D187F0212675822CC
:026226008D5E8B
:10622800EFD3941D402AEF9432502574E22FFFE4F7
:10623800FEEEFD3395E0FCEF75F007A42450F582DF
:10624800E4340A120E3FE4F00EBE07E5D22C8002B9
:07625800C22CAF5E126F1FA4
:01625F00221C
:062D8E008E5E8F5F8D6078
:102D9400D22B120EE5FFE55F2404120DA7122EB507
:102DA400C39418501C855F82855E83A3A3A3E0FFB0
:102DB400E55F2404120DA7FD126DFE7882A607803C
:102DC40006E47882F6C22B120D96122EB5C3943CFB
:102DD400500D120D96FD126DFE7883A6078006E451
:102DE4007883F6C22BE55F2407120DA7FF126EB19C
:102DF4008F61E561D394004017E56194085011E5B3
:102E04005F2407120DA7FF126EB1787FA607800614
:102E1400787F7601C22BE55F2408120DA7FFE55FDA
:102E24002409120DA7122EBE401FE56194205019EB
:102E3400E55F2408120DA7FFE55F2409120DA7FD25
:102E4400126DFE7887A607800678877601C22BE587
:102E54005F240A120DA7FFE55F240B120DA7122EA3
:102E6400BE401FE561940D5019E55F240A120DA7B9
:102E7400FFE55F240B120DA7FD126DFE7880A607F7
:102E8400800678807601C22BE55F240C120DA7FF23
:102E9400E55F240D120DA7FD126DFE7881A60730A3
:102EA4002B07125990D22C8002C22CAF60126F1FD4
:102EB40022FD1264F08F61E56122FD1264F08F61DE
:062EC400E561D394002239
:0653F9008E5E8F5F8D60E7
:1053FF00D22B120EE5FFE55F2404120E6D125464DA
:10540F009418501C855F82855E83A3A3A3E0FFE5FC
:10541F005F2404120E6DFD126DFE7882A6078006C2
:10542F00E47882F6C22B120E5C125464943C500D39
:10543F00120E5CFD126DFE7883A6078006E478835A
:10544F00F6C22B302B07125990D22C8002C22CAFF0
:04545F0060126F1F49
:0B54630022FD1264F08F61E561C3229E
:106EB100120EC54008EF6480948A5001227F00229F
:106DFE00AE05126EB1EFC454F0FDAF06126EB1EFD8
:036E0E004DFF2213
:1063E7008F5ED22D125A997D1E7F081267587D261F
:1063F7007F081267587D527F04126758C22B1269B3
:1064070012125D02787FE6FF125B3C125A43C22DDF
:06641700AF5E125A99224B
:1067FE008D5EEFD3940A4006EFD3940F4003EF70F3
:10680E000E90002BEFF0D22CAF5E126F1FD322C270
:08681E002CAF5E126F1FC322B4
:0255C0008F5EFC
:1055C200D22D125A997D207F051267587D2E7F03B6
:1055D2001267587D527F0412675890002BE0F55FE6
:1055E200E55FB40B067D5F7F078034E55FB40C0690
:1055F2007D5E7F068029E55FB40D067D0A7F02800D
:105602001EE55FB40E067D327F028013E55FB40FA4
:10561200067D467F028008E55F70077D0A7F0312E0
:095622006758C22DAF5E125A99BF
:01562B00225C
:106C42008D5E120EC5400EEF64809486500712646A
:0D6C520088D22C8002C22CAF5E126F1F2270
:026938008D5E72
:10693A00120ECC1264F0120EC54010EF648094A1BE
:10694A005009900029EFF0D22C8002C22CAF5E12BF
:02695A006F1FAD
:01695C002218
:02695D008D5E4D
:10695F00120ECC1264F0120EC54010EF648094A199
:10696F005009900028EFF0D22C8002C22CAF5E129B
:02697F006F1F88
:0169810022F3
:106E1100D3EF648094814008EF6480948A5001220A
:036E21007F0022CD
:106EC100120EC54008EF648094A15001227F002278
:0814D7008E5E8F5F8D608B615A
:1014DF00120EE514F56374FC2561F5616403600F6A
:1014EF00E56164076009E561640B60030216C2C31E
:1014FF00E5636480948050030216C2E563648094B0
:10150F008840030216C2E4F562120D6F7803C333ED
:10151F00CE33CED8F92430F58274003EF583AF6216
:10152F00EF3395E0FE120DEAE4F00562E562B408D0
:10153F00D8756204E56164037029120D4B12170808
:10154F00120D6D7803C333CE33CED8F9120D40A3ED
:10155F00A3120D687803C333CE33CED8F9120FCF51
:10156F000216B9E56164077069120D4B1217081264
:10157F000D6D7803C333CE33CED8F9120D40A3A32C
:10158F00120D687803C333CE33CED8F9120FCF12B2
:10159F000D46A3A3A3120D687803C333CE33CED861
:1015AF00F92432F5827400120D461216CAC333CED7
:1015BF0033CED8F92433F5827400120D46120D5D27
:1015CF007803C333CE33CED8F92434F582740002B6
:1015DF0016B9E561640B60030216C2120D4BE012DF
:1015EF000F00A3E0FD1264F0126EC1120D6D7803AF
:1015FF00C333CE33CED8F9120D40A3A3120D6878A2
:10160F0003C333CE33CED8F9120FCF120D46A3A397
:10161F00A3120D687803C333CE33CED8F92432F535
:10162F00827400120D461216CAC333CE33CED8F9C8
:10163F002433F5827400120D46120D5D7803C33307
:10164F00CE33CED8F92434F5827400120D46E582DC
:10165F002407120D617803C333CE33CED8F9243566
:10166F00F5827400120D46E5822408120E1F120F28
:10167F0000E5822409120E1FFD1264F0126EC112D2
:10168F000D6D7803C333CE33CED8F92436F582747B
:10169F0000120D46E582240A120D617803C333CE82
:1016AF0033CED8F92437F58274003EF583EDF0D2AE
:0A16BF002C8002C22CAF60126F1FD6
:1016C90022E5822404F582E43583F583E0FFE562AF
:1016D900FD3395E0FCE55F2DF582E55E3CF583E59C
:1016E900822405F582E43583F583E0FD1264F01266
:1016F9006EC1AD07AF63EF3395E0FEEF780322E0EB
:10170900FFE562FD3395E0FCE55F2DF582E55E3C82
:0C171900F583A3E0FD1264F0126EC12203
:045D96008D5EAC076B
:105D9A00D3EC648094804035EC64809489502EE47E
:105DAA00FDECFF3395E0FEEF7803C333CE33CED854
:105DBA00F92428F58274003EF583EDFF3395E0FE61
:105DCA00120DEAE4F00DBD08D8D22C8002C22CAF25
:045DDA005E126F1FC7
:015DDE0022A2
:106343008D5E120EC5402FEF648094895028EF14A0
:10635300FFE55E24FF922B125081D22DAF5E125ABD
:10636300997542017F327E00126CEEE54270FCC2E9
:076373002DAF5E125A9922C2
:084683008F5E8C5F8D608B617E
:10468B00856082855F83120E12FD1264F08F62E5E6
:10469B0062D394005003024730E562943340030227
:1046AB004730E55E64067036D22DAF61125A997DA4
:1046BB00527F05126758AF621235B8120F2EB40134
:1046CB000A120E867401F07D388007120E86E4F014
:1046DB007D367F06126758C22DAF61025A99E5608D
:1046EB002406120F32640B703C120F2EB401081209
:1046FB000E867401F08005120E86E4F074F9255EC7
:10470B00F55E75F004123998AFF0EF7014E5602484
:10471B0006FBE4355FFAAD62E4FF1234B8D22C80AD
:0C472B0006C22C8002C22CAF61126F1F6E
:01473700225F
:083004008F5E8C5F8D608B6113
:10300C00856082855F83120E12FD1264F08F62E57B
:10301C0062D394005003023130E5629429400302DC
:10302C003130E55E64067037D22DAF61125A997D4E
:10303C00527F05126758AF621235B8120EB9E0B460
:10304C00010A120E927401F07D388007120E92E480
:10305C00F07D367F06126758C22DAF61025A99E592
:10306C00602406120EBDE0640B6003023130120EB8
:10307C00B9E0B40108120E927401F08005120E92A0
:10308C00E4F0E4FFFEE5602407120EBDE5822E128B
:10309C000E1FB40B04AF0680040EBE08E8EF7003DD
:1030AC00023130C39408507C120F3BEFF07E01EFDD
:1030BC002401FDE433FCEEC39DEC6480F87480982D
:1030CC005020E5602406120EBDE5822E120E1FFD67
:1030DC00120F3BE5822EF582E43583F583EDF00E7D
:1030EC0080CDE5602408120EBDE5822F120E1F6400
:1030FC000B602DEF2408FEC3E55E9EF55E75F004B3
:10310C00123998AEF0EE701CE5602407FDE4355FD3
:10311C00FC7E00ED2FFBEE3CFAAD627F011234B861
:0B312C00D22C8002C22CAF61126F1F7A
:013137002275
:0834B8008F638D648A658B6649
:1034C000756801E4F567120DB4E0FF6409703E12FF
:1034D00035A98003120F13D8FB120DB012359B785B
:1034E00008EF088003120F13D8FB120DB0A3A3E05E
:1034F000FFE568FD3395E0FCE5662DF582E5653C6A
:10350000F583A3A3A3E0FD126E36023554120DB469
:10351000E0FF1235A98003120F13D8FB120DB01271
:10352000359B7804EF088003120F13D8FB120DB0FF
:10353000A3A3E0FF126F80EF426AAE69AF6A78041E
:10354000EF088003120F13D8FB120DB0A3A3A3E062
:10355000FF126F80EF426AE563700FAF67120D7163
:10356000120EAFE564900AC08012E563B40117AF94
:1035700067120D71120EAFE564900530120DE7E58C
:1035800069F0A3E56AF074042568F5680567C3E58A
:0A359000676480949050030234C673
:10359A0022A3E0FF126F80EF426AAE69AF6A22127D
:0E35AA006F807569008F6AAE697804EF0822A1
:0A6F8000EFD3940940037F002222A2
:023A84008B5E57
:103A86001264F08F61E561D394005003023B66E552
:103A96006194334003023B66D22DAF5E125A997D84
:103AA600527F05126758AF611235B8746F256112DF
:103AB6000E96E060047D3880027D367F06126758D8
:103AC6007F2C7E01126CEEE561120F3DE0F55F7012
:103AD600077D1B7F061267587D577F02126758E5E0
:103AE6005F603B756001AF5F120D712401FFE43E1C
:103AF600FEAD60ED3395E0FCC3ED9FEE6480F8EC1F
:103B06006480985019120DD8E0B40A04E4FD8006CA
:103B1600120DD8E0FDE4FF126758056080C87F2CBF
:103B26007E01126CEEE561900530120F899000005F
:103B3600EEF0A3EFF04E70077D1B7F061267587DEF
:103B46000C7F03126758900000E07002A3E0600942
:103B5600E56114FD7F01122AF0C22DAF5E025A996B
:073B6600C22CAF5E126F1FBD
:013B6D002235
:024DD2008B5EF6
:104DD4001264F08F5FE55FD394004077E55F94330E
:104DE4005071D22DAF5E125A997D527F05126758C9
:104DF400AF5F1235B8749F255F120E8AE060047DA0
:104E04003880027D367F061267587F2C7E01126C33
:104E1400EE7F2C7E01126CEEE55F900AC0120F89C2
:104E2400900000EEF0A3EFF04E70077D1B7F06129A
:104E340067587D0C7F03126758900000E07002A34E
:104E4400E06009E55F14FDE4FF122AF0C22DAF5EB5
:0A4E5400025A99C22CAF5E126F1FC4
:014E5E002231
:026260008B5E53
:106262001264F0AD07EDD394004025ED9433502035
:10627200E4FC120EA8ED900AC0120DE7E4F0A3F0C0
:106282000CBC10EE749F2D120E8AE4F0D22C800208
:07629200C22CAF5E126F1F6A
:0162990022E2
:025B8B008B5E2F
:105B8D001264F0AD07EDD394004036ED94335031EF
:105B9D00E4FC120EA8ED900530120DE7E4F0A3F031
:105BAD000CBC10EE746F2D120E96E4F0FCECFF336E
:105BBD0095E0FEED120DE1E4F00CBC08F0D22C8066
:085BCD0002C22CAF5E126F1F33
:015BD50022AD
:042AF0008F628D6301
:102AF400E4F564E5627052AF64120D7125E0FDEEF9
:102B040033FCAF63120D717805C333CE33CED8F9DD
:102B1400120E38120F958003120F1AD8FB120F757C
:102B24008003120F1AD8FB540FF566AF63120D71B0
:102B34007805C333CE33CED8F9120E38120FA180E4
:102B440003120F1AD8FB022BAEE56264017064AF66
:102B540064120D7125E0FDEE33FCAF63120D717844
:102B640005C333CE33CED8F92450F5827405120E42
:102B74003E120F958003120F1AD8FB120F758003B3
:102B8400120F1AD8FB540FF566AF63120D71780556
:102B9400C333CE33CED8F92450F5827405120E3ED9
:102BA400120FA18003120F1AD8FB540FF567ED54CE
:102BB4000FF568E565700CE5667008E5677004E577
:102BC40068607CAD65E4FF126758AD66E4FF126788
:102BD40058E56564097045856769AF69FE7804EF57
:102BE400088003120F13D8FBF569E5684269E569AB
:102BF400B4990B7D09E4FF1267587D098027E569C4
:102C040075F00A84F56AFDE4FF126758E56A75F009
:102C14000AA4FFC3E5699FF56AFD8009AD67E4FF77
:102C2400126758AD68E4FF1267587FF47E01126C96
:0F2C3400EE0564C3E564648094A05003022AF7A0
:012C4300226E
:1064F000EFD394004015EF940B5010EFC3940A5063
:1065000008EF75F00AA4FE8002E4FEEDD39400408B
:106510000EED940B5009EDC3940A5003ED2EFEAF1F
:016520000674
:016521002257
:0649D3008E5E8F5F8B6019
:1049D900756105756240D3ED64809484407CED6413
:1049E9008094A55075ED24FDF563D39404406BE5DF
:1049F9006320E06613F5640562E562AE6170020545
:104A09006114F5828E83E564F07403255FF55FE434
:104A1900355EF55EE4F563E563C395645033855F00
:104A290082855E83E0FFA3E0FD126E360562E562D2
:104A3900AC617002056114F5828C83EFF0055FE5C6
:104A49005F7002055E055FE55F7002055E056380C4
:104A5900C6D22CAF60126F1FD322C22CAF60126F67
:024A69001FC369
:014A6B002228
:043E13008C5F8D60D3
:103E1700120EC55003023EEBEF64809495400302F7
:103E27003EEBEB648094875003023EEBEB64809497
:103E3700E44003023EEB120D717805C333CE33CE57
:103E4700D8F9120FD6F5638F64EB24FBF565D3948D
:103E5700025003023EEBE56575F00384E5F060036D
:103E6700023EEBE56575F00384F567C39410507463
:103E7700120F827002056314F5828E83E567F07472
:103E870005120FE0E4F565E565C395675052120F1B
:103E9700EAE0F566B40A10120F827002056314F5A2
:103EA700828E83E4F0800F120F827002056314F58F
:103EB700828E83E566F0120FEAA3E0FF120FEAA3F2
:103EC700A3E0FD126E368F66120F8270020563142F
:103ED700F5828E83E566F07403120FE0056580A70F
:0B3EE700D22C8002C22CAF62126F1FB1
:013EF20022AD
:0826A8008E5E8F5F8D608B6177
:1026B000C22B120FF160030227451228205003029B
:1026C0002740E5649408E56394075074C3E56064AB
:1026D00080948A506B120EEEA3E0F562B40106906E
:1026E0000520022795E562B402069005220227958F
:1026F000E562B40306900524022795E562B404065A
:10270000900526022795E562B40506900528022764
:1027100095E562B4060690052A022795E562B4079E
:102720000690052C022795E562B4080590052E80D9
:1027300064E562B40905900530805AD22B02281155
:10274000D22B022811120EEEE064017052AD60AF80
:102750005FAE5E1228205003022811E5649408E55C
:102760006394074003022811C3E5606480948A40A3
:1027700003022811120EEEA3E0F562B40A059005DB
:10278000328012E562B401059005348008E562B438
:102790000209900536E563F0A3806FD22B80721298
:1027A0000EEEE06402706AAD60AF5FAE5E125BD6A3
:1027B0007563008F64C3E5649463E56394005051CE
:1027C000C3E560648094885048120EEEA3E0F56281
:1027D000B40107900538EFF08037E562B402059048
:1027E00005398026E562B4030590053A801CE56250
:1027F000B4040590053B8012E562B4050590053CE4
:102800008008E562B4060890053DE564F08002D2D8
:0F2810002B302B04C22C8002D22CAF61126F1F11
:10281F002212488C8E638F64D3E564943BE56394F6
:02282F00002285
:06488C008E658F66A90590
:104892007D057C00120FB9E0C3940A4005120FB9DE
:1048A200E4F00DBD00010CED640A4C70E7B9060797
:1048B200120DF5FF7E0022E964077010120DF575E6
:1048C200F00AA4ACF0FDE5662406801BE9640870DA
:1048D20021120DF575F064A4ACF0FDE56624061214
:1048E2000DF9120F212407120DF92DFDE43CAF053D
:1048F200FE22E964097033120DF5FF7E007C037D10
:10490200E81239BAAC06AD07E5662406120DF97550
:10491200F064120F242407120DF9120F2124081239
:0D4922000DF92DFDE43CFEAF0522E4FEFF83
:01492F002265
:065BD6008E658F66A90533
:105BDC007F057E00120FC4E0C3940A4005120FC467
:105BEC00E4F00FBF00010EEF64084E70E7E96407A4
:105BFC007020E5662405F582E43565F583E075F0E3
:105C0C000AA4FFE5662406F582E43565F583E02FEA
:045C1C00FF227F00E4
:015C20002261
:083391008E5E8F5F8D608B6181
:10339900C22BD3E56064809484500302343FE56016
:1033A9006480948D400302343F120FF160030234AC
:1033B9003F120EE5123A5E33DF0133EA0233F503B9
:1033C90033FF04340905341306341D073427083440
:1033D90031090000343B756201756300D22B023458
:1033E90076756201756308D22B02347675620175B0
:1033F9006310D22B8077756201756318D22B806DAB
:10340900756201756320D22B80637562017563282B
:10341900D22B8059756201756330D22B804F75624A
:1034290001756338D22B8045756201756340D22BD3
:10343900803BC22B8037D3E56064809484402EE5BD
:10344900606480948D5026855F82855E83A3A3E0A6
:10345900B4011A855F82855E83A3A3A3E024F67075
:103469000A756201756358D22B8002C22B302B3743
:10347900E4FF120F60E4F00FBF08F7E56024FB8555
:103489006382856283F07F01E55F2404F582E43578
:103499005EF583E5822F120E1FFE120F60EEF00F0C
:0E34A900BF08E5D22C8002C22CAF61126F1F4B
:0134B70022F2
:044738008F5E8D5FA4
:10473C00E55ED3940050030247DBE55E941540031D
:10474C000247DBD22DAF5F125A997D5F7F0512674E
:10475C0058AD5EE4FF1267587D527F041267587F94
:10476C00F47E01126CEE75F020E55E900280123A38
:10477C0052AF828583628F63E0F560603DD3940015
:10478C004046E56094105040E56025E0F5607561A9
:10479C0001E5602401FFE433FEC3E5619FEE648014
:1047AC00F87480985022120FADE0FF120FADA3E009
:1047BC00FD1265E50561056180D77D1B7F061267DB
:1047CC00587D5F7F05126758C22DAF5F025A99C2A0
:0647DC002CAF5F126F1FFD
:0147E20022B4
:10216D008F5E8D5F8B60E55E640A7074E55FC3946E
:10217D000A40030222DA122310E4FDFF126758AD64
:10218D005F1222E9E55F123A5E21B50121BB022102
:10219D00C10321C70421CD0521D30621D90721DF94
:1021AD000821E509000021EA90052002223490055E
:1021BD002202223490052402223490052602223474
:1021CD0090052802223490052A02223490052C0213
:1021DD00223490052E022234900530804A0222D3FB
:1021ED00E55E64017052E55FD394004006E55F94AF
:1021FD00034006E55F640A703C122310E55FB40AE4
:10220D000A7D0A1222E9900532801CE55FB4010AAD
:10221D007D0B1222F6900534800DE55FB402137D1F
:10222D000C1222F6900536E0FEA3E0FF1265540273
:10223D0022E10222D30222DAE55E64026003022269
:10224D00E1E55FD3940050030222DAE55F94075075
:10225D007CD22DAF60125A997D277F081267587D69
:10226D0006E4FF1267587D14E4FF126758E55F24FA
:10227D00FE601A14602114602814602F1460362437
:10228D000570437D0112230390053880307D0212C5
:10229D00230390053980267D0312232690053A806D
:1022AD001C7D0412232690053B80127D05122333DD
:1022BD0090053C80087D0612233390053DE0FF7E9E
:1022CD0000126585800EAF60126C5F8007C22CAF67
:1022DD0060126F1FC22DAF60125A9922E4FF126770
:1022ED00587D527F0412675822E4FF1267587D52C1
:1022FD007F0412675822E4FF1267587D527F041243
:10230D00675822D22DAF60125A997D277F08126728
:10231D00587D06E4FF12675822E4FF1267587D527C
:10232D007F0412675822E4FF1267587D527F041212
:03233D00675822BC
:044B04008E638F64C9
:104B08000564E5647002056314F5828E83E0F5663A
:104B1800607AC3940850757F2C7E01126CEEE4F520
:104B280065E565C395665064856482856383E01294
:104B38003A5E4B75004B530A4B570B4B5D0C4B635E
:104B48000D4B690E4B6F0F00004B7BE4FD802D7DF4
:104B58005F7F0780287D5E7F0680227D0A7F028036
:104B68001C7D327F0280167D467F0280107D0A7F81
:104B780003800A856482856383E0FDE4FF12675839
:0C4B88000564E564700205630565809516
:014B940022FE
:061F7B008F5E8D5F8B609C
:101F8100C22BE55E640A600302206FE55F123A5ED0
:101F91001FB0011FC3021FD6031FE9041FFC052048
:101FA1001206202807203E082053090000206B124A
:101FB10020A47D011220F2756101756200D22B020D
:101FC100208B1220A47D021220F275610175620836
:101FD100D22B02208B1220C07D031220FF756101DC
:101FE100756210D22B02208B1220C07D041220FFBB
:101FF100756101756218D22B02208B1220DC12212F
:10200100527D05122122756101756220D22B0220B9
:102011008B1220DC1221527D06122122756101757D
:102021006228D22B02208B12210C1221667D07120D
:10203100212F756101756230D22B02208B12210C88
:102041001221667D0812212F756101756238D22B2C
:10205100803812213CE4FDFF1267587D0912215995
:10206100756101756240D22B8020C22B801CE55E18
:1020710064017016E55F24F6701012213C7D0A128E
:102081002159756101756258D22B302B09AF62AEAF
:1020910061124B048005AF60126C5FC22DAF6012FC
:0220A1005A994A
:1020A30022D22DAF60125A997D577F021267587D55
:1020B30005E4FF126758E4FDFF12675822D22DAFE3
:1020C30060125A997D577F021267587D05E4FF120B
:1020D3006758E4FDFF12675822D22DAF60125A9958
:1020E3007D577F021267587D05E4FF12675822E48B
:1020F300FF1267587D527F0412675822E4FF12676C
:10210300587D527F0412675822D22DAF60125A991C
:102113007D577F021267587D05E4FF12675822E45A
:10212300FF1267587D527F0412675822E4FF12673B
:10213300587D527F0412675822D22DAF60125A99EC
:102143007D577F021267587D05E4FF12675822E42A
:10215300FDFF12675822E4FF1267587D527F041275
:0A216300675822E4FDFF12675822BE
:1035B8008F72E572D3945940107D5A12369F24A613
:1035C800FD700302369E023699E572D3944F401679
:1035D800E572945A50107D5012369F24B0FD700346
:1035E80002369E023699E572D394454016E57294E8
:1035F8005050107D461236A724BAFD700302369E3D
:10360800023699E572D3943B4012E5729446500C09
:103618007D3C1236A724C4FD607C8075E572D39486
:10362800314012E572943C500C7D321236AF24CEF4
:10363800FD6063805CE572D394274012E572943292
:10364800500C7D281236AF24D8FD604A8043E572BD
:10365800D3941D4016E572942850107D1EE4FF1285
:103668006758E57224E2FD602D8026E572D3941335
:103678004016E572941E50107D14E4FF126758E559
:103688007224ECFD60108009E572C394145007ADF4
:1036980072E4FF12675822E4FF126758E57222E4C9
:0F36A800FF126758E57222E4FF126758E572229D
:105A99008F6AE56A700C302D097F01126F9D7FC0F6
:105AA900801FE56A700C202D097F01126F8A7FC063
:105AB9008026E56AB40112302D0F7F02126F9D7F97
:105AC90030120016C22F026A14E56AB40114202D9F
:105AD900117F02126F8A7F30126F497FC87E0012D0
:035AE9006CEE223E
:1069F0008F69D22D125A997D607F021267587D32BD
:106A00007F061267587D1E7F05126758C22DAF6939
:046A1000125A99225B
:106C5F008F69D22D125A997D607F021267587D304D
:0D6C6F007F03126758C22DAF69125A992297
:0E6F1F008F68302C030269F0AF68126C5F229D
:105E2800EF24FE60101460162402701C7F01126FAC
:105E38009D7F8080107F02126F9D7F2080077F03E7
:105E4800126F9D7FA01200167FF47E01126CEE7512
:105E58004204E54270FC7F647E00126CEE7F031200
:085E68006F8A7FA0126F49222E
:106585008E618F627C007D0A1239CCAD07E4FF1263
:1065950067587D5B7F06126758AE61AF627C007DF0
:1065A5000A1239CCE4FF1267587D4A7F0702675803
:046554008E618F6263
:106558007C007D3C1239CC1235B87D057F06126768
:1065680058AE61AF627C007D3C1239CCED4C600CBA
:0C657800AF051235B87D4A7F0712675846
:0165840022F4
:02607F008D5E34
:10608100120EC5402FEF648094955028120D71783F
:1060910005C333CE33CED8F9120FD6FEE4FD0FEF90
:1060A100AA0670010E14F5828A83E4F00DBD20EE7C
:0B60B100D22C8002C22CAF5E126F1FC9
:0160BC0022C1
:1060FB008F5E900540E0D394024015D22D125A9931
:10610B007542037F327E00126CEEE54270FC801507
:10611B00D22DAF5E125A997D1B7F061267587D0CEC
:0D612B007F03126758C22DAF5E125A9922F1
:106E24007E10900540E4F0A3DEFC7E10D22C126F9D
:016E34001F3E
:016E3500223A
:106E3600BF0A02E4FFBD0A02E4FDEF75F00AA42DC5
:026E4600FF2229
:106CB600EFD394094002E4FFEDD394094002E4FDCA
:0C6CC6007804EF08800123D8FD4DFF2268
:10409D0007010203040506070707060504030201CD
:1040AD0003010A0A030307050303020503020A0AB3
:1040BD0004050A0A0104050A0A0A04050A0A02038C
:1040CD00070A0A03040A0A04024B00020032072EF3
:1040DD0003024B0002003202055F000302055F0080
:1040ED000402055F000502055F000604072E082681
:1040FD000640033204072E08260640025304081E0C
:10410D0008260452010008024B00020032072E0857
:10411D001E08260452010003072B0235063603073D
:10412D002B0235063803072B0235072603072B0212
:10413D0035025302055F000F02055F001002055F97
:10414D00001102055F001202055F001302055F00FA
:0A415D0014080C0A1D020500241BC3
:105380007461F0A37420F0A37452F0A37401F0A32D
:1053900022A3F0A37461F0A37440F022F0A374037D
:1053A000F0E4A3F0A37410F0A37403F0E4A3F0A35B
:1053B000227461F0A37441F0A3227461F0A3F0A3FE
:1053C0007430F0A3227496F0A37432F0A37495F0B5
:1053D000A3741EF0A322F0A37461F0A314F0A374CD
:1053E00070F0A3E4F022A3F0A37452F0A3223CF5E2
:0953F00083E0FEEF3395E0FC229E
:10003E007E407F9D7C017D507B08125F7D7E407FE0
:10004E00A57C017D587B08125F7D7E407FAD7C01D3
:10005E007D007B04125F7D7E407FB97C017D087B35
:10006E0004125F7D7E407FB57C017D107B04125FA4
:10007E007D7E407FB17C017D187B04125F7D7E40CA
:10008E007FC27C017D207B05125F7D7E407FBD7C23
:10009E00017D287B05125F7D7E407FC77C017D3010
:1000AE007B05125F7D7E407FCC7C017D387B041208
:1000BE005F7D7E407FD07C017D407B04125F7D7E24
:1000CE00407FD47C027DA07B09125F7D7E407FDD68
:1000DE007C027DC07B07125F7D7E407FE47C027DCB
:1000EE00E07B05125F7D7E407FE97C037D007B0512
:1000FE00125F7D7E407FEE7C037D207B05125F7D4F
:10010E007E407FF37C037D407B05125F7D7E407FCA
:10011E00F87C037D607B09125F7D7E417F017C034D
:10012E007D807B09125F7D7E417F0A7C037DA07BF3
:10013E0009125F7D7E417F137C037DC07B11125FB0
:10014E007D7E417F247C037DE07B07125F7D7E41B7
:10015E007F2B7C047D007B07125F7D7E417F327C8E
:10016E00047D207B07125F7D7E417F397C047D40BC
:10017E007B07125F7D7E417F407C047D607B051294
:10018E005F7D7E417F457C047D807B05125F7D7E99
:10019E00417F4A7C047DA07B05125F7D7E417F4FAF
:1001AE007C047DC07B05125F7D7E417F547C047D87
:1001BE00E07B05125F7D7E417F597C057D007B05CE
:1001CE00125F7D7E417F5E7C057D407B09125F7DE7
:1001DE009000297417F07F03126488900028741918
:1001EE00F090002074B1F09000217491F0900022F4
:1001FE007403F0900023747FF090002404F09000BC
:10020E00257403F0E4900026F0900027F090003063
:10021E00740912539C7415F0A37403F0A374151291
:10022E00539C7409F0A37403F0E4FFEFFD3395E0E3
:10023E00FC74302DF58274001253EE74102DF5827D
:10024E0074003CF583EEF00FBF08E0E4FFEFFD33E2
:10025E0095E0FC74382DF58274001253EE74182D4F
:10026E00F58274003CF583EEF00FBF08E090052098
:10027E00E4F0A374B4F0900522E4F0A374B4F0900B
:10028E0005247401F0A374E0F0900526E4F0A37445
:10029E0078F09005287402F0A37458F090052AE4C3
:1002AE00F0A3743CF090052C7402F0A37458F07413
:1002BE000790052EF0A3F0900530F0A3F0900532D4
:1002CE00F0A3F0900534F0A3F0900536E4F0A3749B
:1002DE003CF0900538740AF09005397428F09005BA
:1002EE003A7405F090053B740AF090053CF09005C9
:1002FE003D7428F09000A47401F0900B607415F01A
:10030E00A37411F09000A57401F0900B807415F099
:10031E00A37410F09000A67401F0900BA07415F069
:10032E00A37421F09000A77401F0900BC07415F027
:10033E00A37420F09000A87401F0900BE07415F0F7
:10034E00A37431F09000A97401F0900C007415F0B4
:10035E00A37430F09000AA7401F0900C207415F084
:10036E00A37441F09000AB7401F0900C407415F042
:10037E00A37440F09000AC7401F0900C60745312B2
:10038E00538A743612538A7438F0A3E4F0A374536C
:10039E00F0A3E4F09000AD04F0900C80745312536F
:1003AE008A7434F0A37421F0A37453F0A3E4F09094
:1003BE0000AF04F0900CC01253887430F074031226
:1003CE0053E6E4F09000B004F0900CE01253887401
:1003DE0030F074041253E6E4F09000B104F0900D86
:1003EE0000125380743212538A7452F0A37420F0A8
:1003FE009000B27401F0900D201253807432F0A36D
:10040E0074021253E77420F09000B37401F0900D53
:10041E0040745312538A7433F0A3E4F09000B40482
:10042E00F0900D601253B17430F07402125391902B
:10043E0000B57401F0900D801253B17430F0740554
:10044E001253919000B67401F0900DA01253B17436
:10045E0030F0A374061253929000B77401F0900D11
:10046E00C01253B11253C57498F0A3744B12539229
:10047E009000B87401F0900DE01253B11253C57490
:10048E0093F0A374181253929000B97401F0900E69
:10049E00001253B17430F0A37413125392A37470FC
:1004AE00F0A37402F09000BA14F0900E201253BA1A
:1004BE007412F0A3747012538A7461F0A314F09046
:1004CE0000BB7401F0900E401253BA74111253D641
:1004DE009000BC04F07461900E601253BC74141240
:1004EE0053D69000D104F09011001253B17492F0D3
:1004FE00A3744BF0A37490F0A37402F0A37490F065
:10050E00A37432F07499A3F0A3F0A3746012538A0B
:10051E00749112538A7491F0A3E412539290000FC7
:10052E007401F0125E707F01126F9D7F40120016F3
:10053E007D2F7F071267587D0C7F031267587D321F
:0C054E007F061267587D1E7F051267585B
:01055A00227E
:0A5F7D008E5A8F5B8C5C8D5D8B5E8D
:105F8700E4F9C3E55E6480F8E96480985028E9FF86
:105F97003395E0FEE55B2FF582E55A3EF583E49302
:105FA700FFE9FD3395E0FCE55D2DF582E55C3CF509
:065FB70083EFF00980CC2D
:015FBD0022C1
:1056FB00AF6AEF3395E0FEE56975F008A42428F551
:10570B0082E43400F583E5822FF582E5833EF58351
:10571B00E0FFE56AFD3395E0FC22AB66AD65AF6457
:10572B00223EF583E0FD74B82FF582741D3EF583A0
:10573B00EDF0056AE56A22EF3395E0FEEF25E0FF19
:10574B00EE33FE22A2E0CE13CE13223CF583EFF014
:05575B00056AE56A2269
:045C21008C5B8D5CAF
:105C2500EF6043D201D202D20CE4F55D855C82853A
:105C35005B83E0FEA3E04E6027AF5D125742E55C53
:105C45002FF582E55B3EF583E0FEA3E0FF1244609D
:105C5500922920290B055DC3E55D6480949040CCB5
:065C6500C201C202C20CE4
:015C6B002216
:045C6C008C608D615A
:105C7000EF6043D201D202D20CE4F56285618285E5
:105C80006083E0FEA3E04E6027AF62125742E561F9
:105C90002FF582E5603EF583E0FEA3E0FF1244604D
:105CA000922D202D0B0562C3E5626480949040CC58
:065CB000C201C202C20C99
:015CB60022CB
:04446000AD07AC06F2
:10446400C22E780CEF08800312574FD8FB540FF577
:10447400637808AF05AE04EF08800312574FD8FBEA
:10448400540FF5647804AF05AE04EF0880031257A7
:104494004FD8FB540FF565ED540FF566E563607175
:1044A400B40108125725123C518066E563B4020832
:1044B400125725126BCA8059E563B40308125725B5
:1044C4001238AA804CE563B40408125725126B6BAA
:1044D400803FE563B405081257251224FA8032E5BB
:1044E40063B406081257251212698025E563B407E0
:1044F4000812572512520A8018E563B408081257A7
:1045040025125935800BE563B40906125725126943
:0345140082A22E52
:014517002281
:103C51008F678D688B69E567B40113900020E0FFE1
:103C61001259EB900020EFF0FD7F20023D0EE56739
:103C7100B40211900021123D14900021EFF0FD7F5C
:103C810021023D0EE567B40311900022123D14900C
:103C91000022EFF0FD7F22023D0EE567B404109093
:103CA1000023123D1E900023EFF0FD7F23805EE58F
:103CB10067B40516900024123D1E900024EFF0FD1C
:103CC1007F247E0012641D0265B5E567B40610907D
:103CD1000025123D28900025EFF0FD7F25802EE57F
:103CE10067B40710900026123D28900026EFF0FDE2
:103CF1007F268019E567B40819900027E0FFAB69BA
:103D0100AD681259EB900027EFF0FD7F277E00127E
:103D1100641D22E0FFAB69AD681259EB22E0FFABF5
:103D210069AD681259EB22E0FFAB69AD681259EB3E
:013D3100226F
:1059EB00D22FAC07BD01047E018033BD02047E02C1
:1059FB00802CBD03047E048025BD04047E08801E1C
:105A0B00BD05047E108017BD06047E208010BD07E7
:105A1B00047E408009BD08047E808002C22FBB013A
:105A2B0005EE4204800BEB7006EEF452048002C2CA
:075A3B002F302F03AF0422FE
:015A42002241
:026BCA008B67D7
:106BCC00C22FEF7016ED7013E5677003025D02E5DE
:0B6BDC0067B40107787FE6FF125B3C06
:016BE700228B
:0638AA008F678D688B6939
:1038B000E5677007123990E4FD801AE567B40107E7
:1038C0001239907D01800EE567B4020CAD69AF68D6
:1038D000126F2D7D02024F72E567B40306124D444C
:1038E000C21E22E567B40415AD69AF681264F08F9B
:1038F00043754205E542700302398F80F7E567643E
:10390000067017E5687013F56A1256FB74102DF5F2
:10391000827400125756B408F022E56764077017E6
:10392000E5687013F56A1256FB74182DF582740061
:10393000125756B408F022E56764087027E56870EE
:1039400023E569701FF56AAF6AEF3395E0FE7410E6
:103950002FF582740012572CB408EC754201E54231
:10396000602D80FAE56764097025E5687021E569D6
:10397000701DF56AAF6AEF3395E0FE74182FF5827B
:0F398000740012572CB408EC754201E54270FC3C
:09398F0022AD69AF68126F2D2210
:106B6B008F67AE03AF05E567D394004012E56794DA
:106B7B0007500CAD06126F2DAD07AF671267AC2235
:1024FA008F678D688B69E5677018E5687014E56900
:10250A0070057F01126F49E569640160030226A71D
:10251A008043E567701CE568B40117E56970057FBB
:10252A0004126F49E569640160030226A77F040269
:10253A0026A4E5677029E56864027023E5697005D9
:10254A007F05126F49E569640160030226A79000BE
:10255A000FE0B403057F010226A47F050226A4E545
:10256A0067B4011BE5687017E56970057F02126F91
:10257A0049E569640160030226A77F020226A4E5F1
:10258A0067B4011CE568B40117E56970057F081294
:10259A006F49E569640160030226A77F080226A441
:1025AA00E56764017029E56864027023E5697005CE
:1025BA007F0A126F49E569640160030226A7900049
:1025CA000FE0B403057F020226A47F0A0226A4E5CF
:1025DA0067B4021BE5687017E56970057F40126FE2
:1025EA0049E569640160030226A77F400226A4E543
:1025FA0067B4021CE568B40117E56970057F10121B
:10260A006F49E569640160030226A77F100226A4C8
:10261A00E56764027024E5686402701EE569700566
:10262A007F50126F49E5696401707290000FE0B43F
:10263A0003047F4080647F508060E567B40317E538
:10264A00687013E56970057F80126F49E569640156
:10265A00704B7F808044E567B40318E568B40113C2
:10266A00E56970057F20126F49E5696401702E7F64
:10267A00208027E56764037024E5686402701EE51C
:10268A006970057FA0126F49E569B4011090000FC7
:0E269A00E0B403047F8080027FA012001622AD
:101269008F678D688B69E5677017AD69AF68126F15
:101279002D8E348F35D3E5359400E534940050F53F
:1012890022E567B4011BE568B40116E5697007C278
:10129900307F01122ECAE569640160030214D68009
:1012A90058E5676401702BE56864027025E569708B
:1012B90007C2307F02122ECAE56964016003021475
:1012C900D690000FE0640370030214D6D2307F0277
:1012D9008031E5676401702EE56864037028E5696B
:1012E9007007C2307F03122ECAE5696401600302E8
:1012F90014D690000FE0B40306D2307F018004D2E7
:10130900307F03022ECAE5676401702DE568640425
:101319007027E569700CC2307F01122ECA7F401216
:101329006F49E569640160030214D6D2307F011266
:101339002ECA7F40120016807CE5676401703AE589
:101349006864057034E569700CC2307F02122ECAD8
:101359007F10126F49E569640160030214D6900099
:101369000FE0640370030214D6D2307F02122ECA32
:101379007F10120016D22F803EE5676401703BE5AD
:101389006864067035E569700CC2307F03122ECA95
:101399007F50126F49E569640160030214D6D230A7
:1013A9007F03122ECA90000FE0B403047F4080022D
:1013B9007F50120016C22F026A14E5676402702971
:1013C900E56864017023E56970057F100214BDE5C5
:1013D90069B401057F100214C7E56964026003025C
:1013E90014D6D22F7F010214D3E56764027029E570
:1013F9006864027023E56970057F200214BDE56900
:10140900B401057F200214C7E56964026003021470
:10141900D6D22F7F020214D3E56764027029E568EA
:1014290064037023E56970057F400214BDE569B462
:1014390001057F400214C7E569640260030214D6FE
:10144900D22F7F030214D3E56764027023E5686431
:1014590004701DE56970047F808059E569B4010451
:101469007F80805AE56964027063D22F7F04805AB5
:10147900E56764027023E5686405701DE569700419
:101489007F048030E569B401047F048031E5696433
:1014990002703AD22F7F058031E5676402702EE52C
:1014A90068640670287D017F07124EEA401FE569CE
:1014B90070057F08026F8AE569B401057F08026F2C
:0E14C9009DE569B40207D22F7F0612299222F8
:06520A008F678D688B69BF
:10521000E567703BE5687037E569700690000F043C
:105220008021E569B4010A90000F7402F0D22F804A
:1052300047E56964027041C21E7FFF126F4990000A
:105240000F7403F0C2307F02122ECAD22F8029E5DC
:105250006764017023E568701F7D077F05124EEAC1
:105260005016E569700BC200C2307F03122ECA804F
:1052700007E569B40102D200302F0C90000FE0FD69
:075280007F0F7E0012641D88
:015287002204
:105935008F678D688B69E567700C125979749F2F95
:10594500F58274008019E567B4010C125979749FCA
:105955002FF58274008016E567B402091259813E5D
:10596500F583E4F022E567B403091259813EF58316
:105975007401F022AD69AF68126F2D22AD69AF6871
:0B598500126F2D746F2FF5827400224A
:026982008F671D
:10698400AF057804EF08800123D8FD4BF568E5676F
:10699400B40908E568B49903024FFAAD68AF671209
:0269A40065E5A7
:0169A60022CE
:0D6F2D00EF75F00AA47C002DFFEC35F0FE9E
:016F3A002234
:0467AC008F688D69FC
:1067B000C3E569648094E4501BE4F56AC3E5696449
:1067C00080F8E56A648098500BC22FAF6812299256
:0467D000056A80E8EE
:0167D40022A2
:0D6F3B00C296007F051268EC126522D29606
:016F48002226
:106DD200126F3BEF20E0F9C296007F061268ECC208
:066DE200B60000D296226B
:106DE800126F3BEF20E0F9C296007F041268ECC2F4
:066DF800B60000D2962255
:0460BD008E608F6101
:1060C100AE04AF058E638F64C296007F031268EC45
:1060D100E560FF1268ECAF611268ECE4F5621265ED
:1060E10022E5642562F582E43563F583EFF005620C
:0960F100E562C3942040E7D29659
:0160FA002283
:085CB7008E658F668C678D6815
:105CBF00126F3BEF20E0F985656A85666BC296002F
:105CCF007F021268ECE567FF1268ECAF681268ECB0
:105CDF00E4F569E56B2569F582E4356AF583E0FF44
:105CEF001268EC0569E569C3942040E7C2B600006D
:025CFF00D2963B
:015D0100227F
:0A5695008E5A8F5B8C5C8D5D8B5E7E
:10569F00C2AF126DD2126F3BEF20E0F9855C6085CF
:1056AF005D61C296007F021268ECE55AFF1268EC4A
:1056BF00AF5B1268ECE4F55FAF5EEF3395E0FEC3CE
:1056CF00E55F9FEE6480F87480985014E561255F64
:1056DF00F582E43560F583E0FF1268EC055F80D852
:0B56EF00C2B60000D296126DE8D2AFE8
:0156FA00228D
:10641D008E6B8F6C8D6DC2AF126DD2126F3BEF20F4
:10642D00E0F9C296007F021268ECE56BFF1268EC92
:10643D00AF6C1268ECAF6D1268ECC2B60000D2966C
:06644D00126DE8D2AF223F
:10613800C2AFE4F55BF55CF55DF55EF55FF55AAE6B
:106148005EAF5FAC5BAD5C1260BD7420255CF55C36
:10615800E4355BF55B7420255FF55FE4355EF55E3D
:0B616800055AE55AC3948940D6D2AF17
:016173002209
:105E7000C2AF756200756300756400E4F560F5619A
:105E8000F55F126DD2AE63AF64AC60AD61125CB70A
:105E900074202561F561E43560F56074202564F5B2
:105EA00064E43563F563055FE55FC3948940D3120D
:045EB0006DE8D2AF18
:015EB40022CB
:1057BF000500050105030507050F051F051E051C3F
:1057CF00051805100201040E040A03060101040B5B
:1057DF000304040F020304010302040D020002027A
:1057EF00030004090404030503070100030304076E
:1057FF00030104060402040C051605150000061526
:0E580F00062A060C06380633061E0612061779
:104CB5002430F58274003EF583EDFF3395E0FEE583
:104CC500822FF582E5833EF583E0FFEDFB3395E02A
:104CD500FA22AF411268ECC293126F94D293D2AF0D
:104CE500223EF583E0FC74B82FF582741D3EF583F2
:104CF500ECF00D221528E528D394002225E024BFE9
:104D0500F582E43457F583E49322E4F57BD20EC2B1
:104D150027C21DC21A227FA0126F49E4F542C21EA6
:104D250022126F94D2B67801EF0822122C44D2CA0F
:0F4D3500D20ED22722ECFF3395E0FEEF78032257
:10416700200E2F900540E004F576D36480948150AB
:1041770003024227D3E5766480948F400375760F58
:10418700900029E0FF122C4490002AE0F575124DAB
:104197000F22301A58302712124CF94003024227D7
:1041A700C2CAC227D21D85752822301D0A124CF9B2
:1041B700506EC227C21D22AF791579EF700BC21A54
:1041C700E57525E0F528D21D22E57A30E0058575ED
:1041D700288008E57575F003A4F528AF7A7801EF14
:1041E70008800103D8FDF57AD227D2CA22D57608EE
:1041F700C20EE4F542C21E22057B7440257BF58280
:10420700E43405F583E0124D01540FF579740193F9
:10421700F57A700AD21DE57525E025E0F528D21A52
:014227002274
:10528800200E12900029E0FF122C4490002AE0F52D
:1052980077124D0F22301A5130270F124CF9505DFA
:1052A800C2CAC227D21D85772822301D0A124CF99E
:1052B800504BC227C21D22AF791579EF7007C21A69
:1052C800C20EF54222E57A30E0058577288008E5A8
:1052D8007775F003A4F528AF7A7801EF0880010309
:1052E800D8FDF57AD227D2CA22E543124D01FA74C5
:0D52F8000193FBEA540FF579EBF57AD21A19
:015305002285
:10652200E4F56FD297F56EC2B6126F94AF6F780131
:10653200EF08800123D8FDF56F309703436F0112F6
:106542006F94D2B6056EC3E56E6480948840D8AF6E
:016552006FD9
:016553002225
:096F9400000000000000000022D2
:10670100C2B7E4FEC2B6126F94EF30E704D2B5808F
:1067110002C2B5124D26800123D8FDFF126F940EDF
:0B672100BE08E1C2B6D2B7D2B6D2B5B6
:01672C00224A
:0D001600C2AFEF4227AF27126701D2AF2221
:0E6F4900C2AFEFF45227AF27126701D2AF227A
:1068EC00E4FEC2B6126F94EF30E704D2B58002C258
:1068FC00B5124D26800123D8FDFF126F940EBE08F1
:05690C00E1D2B6D2B596
:016911002263
:096F9D00C2AFEF4241124CD722B1
:0A6F8A00C2AFEFF45241124CD722BF
:102C4400EF123A5E2CAC012CB3022CBA032CC10453
:102C54002CC8052CCF062CD6072CDD082CE4092C17
:102C6400EB0A2CF20B2CF90C2D000D2D070E2D0E5A
:102C74000F2D15102D1C112D23122D2A132D311457
:102C84002D38152D3F162D46172D4D182D54192D61
:102C94005B1A2D621B2D691C2D6B1D2D721E2D7947
:102CA4001F2D802000002D6975CB8E75CAC6227534
:102CB400CB9575CA772275CB9B75CA692275CBA053
:102CC40075CABA2275CBA675CA332275CBAB75CA41
:102CD400632275CBB075CA022275CBB475CAA32220
:102CE40075CBB875CAFA2275CBBC75CAD82275CB18
:102CF400C075CAA82275CBC475CA362275CBC775F0
:102D0400CA862275CBCA75CABC2275CBCD75CAB426
:102D14002275CBD075CA762275CBD375CA3022758D
:102D2400CBD575CAB22275CBD875CA132275CBDA46
:102D340075CA522275CBDC75CA7D2275CBDD75CA86
:102D44006E2275CBE075CA542275CBE275CA1B227C
:102D540075CBE375CAC32275CBE575CA5E2275CB04
:102D6400E675CADA22801C75CBE875CA902275CB49
:102D7400EA75CAD92275CBEC75CA092275CBED75F3
:0A2D8400CA292275CBE875CA412266
:10002600C3EF648094A15008EF25E025E0F528226F
:04003600E4F52822A3
:0237B3008F5A2B
:1037B500900118E0FFE55A7006E545D39F5012E5E4
:1037C5005A640160030238A9E546D39F50030238C5
:1037D500A9E55A7018C3E5459FF55D74602FF5821C
:1037E500E4341EAD82F55E8D5F7F40801BE55AB4E3
:1037F5000119C3E5469FF55D74B02FF582E4341ECB
:10380500AF82F55E8F5F7F101200167FF47E011286
:103815006CEE7D207F051267587D1A7F0812675868
:103825007FC87E00126CEEE4F55BE55BC3955D50E9
:1038350061055FE55FAE5E7002055E14F5828E83FD
:10384500E0F55C123A5E38860038640A38680B3851
:103855006E0C38740D387A0E38800F0000388CE401
:10386500FD80277D5F7F0780227D5E7F06801C7D32
:103875000A7F0280167D327F0280107D467F02809E
:103885000A7D0A7F038004AD5CE4FF126758055B7F
:103895008098E55A70047F408007E55AB401057F9A
:0438A50010126F4945
:0138A90022FC
:10510700200E10754406901DB8E06003D20E22E40D
:10511700F54222E528D394004003152822C2CA1578
:1051270044E54414603D14603214601D1460151486
:105137007049901DB8E0FF7003F54222122C44908D
:105147001DB9802F901DBA8015901DBBE0FF70031D
:10515700F54222122C44901DBC8018901DBDE0FF23
:10516700020026901DBEE0FF7003F54222122C4478
:10517700901DBFE0FF120026D2CA22E4F542C2CA40
:03518700C20E2233
:1066D300900028E0FF6026200E07124D3075281425
:1066E30022E528D394004003152822202708D2CA84
:0E66F300752814D22722C2CA75287DC227221C
:10667500200E0C7F1C124D3075286475783C22E580
:1066850028D394004003152822AF781578D3EF64FA
:0E669500809480400475286422C20EE4F54211
:0166A30022D4
:10637A00E54214601C14601C14601F14602214602F
:10638A002224057021C2CAC20EC227C21DE4F544E6
:10639A00220251071266D3D21E22124167D21E224E
:0763AA000266751252882201
:10648800BF010790002A7418F022BF020790002A63
:106498007412F022BF030590002A8014BF040790ED
:1064A800002A740BF02290002ABF05047409F02218
:0464B800740CF0224E
:02508100AC077A
:10508300C3EC64809480404AEC648094885043204D
:105093002B21E4FD124D3AC333CE33CED8F9124C53
:1050A300B574102BF58274003AF583EFF00DBD084B
:1050B300E3801FE4FD124D3AC333CE33CED8F91249
:1050C3004CB574182BF58274003AF583EFF00DBDDF
:1050D30008E3202B16E4FDEDFF3395E0FE74102F5B
:1050E300F5827400124CE6BD08ED22302B15E4FD69
:1050F300EDFF3395E0FE74182FF5827400124CE631
:03510300BD08EDF7
:015106002286
:104FFA007D3F7F091267587D507F08126758906F6E
:10500A00C61250787D5B7F06126758906FC71250A0
:10501A0078906FC8E493FDE4FF126758906FC9E473
:10502A0093123A5E504A41504E42505243505844AD
:10503A00505E45506446506A4750704800005077A9
:10504A007D0A80067D3280027D467F02801C7D0AB1
:10505A007F0380167D287F0380107D467F03800AA8
:10506A007D0A7F0480047D287F0412675822E49316
:07507A00FDE4FF126758225C
:105FFF008F5BE55B7005D22DFF8009E55BB4010770
:10600F00D22D7F01125A997D4B7F021267587D0264
:10601F00E4FF1267587D32E4FF126758124FFAE51A
:10602F005B70028005E55BB401057F40126F49226A
:103D3200A209300501B350307D017F04124EEA50D2
:103D42002320050E30090B9000A4E0FF7C0B7D6060
:103D5200800F30050F20090C9000A5E0FF7C0B7D41
:103D620080125C6CA2099205A20A300601B350309F
:103D72007D027F04124EEA502320060E300A0B9079
:103D820000A6E0FF7C0B7DA0800F30060F200A0CFE
:103D92009000A7E0FF7C0B7DC0125C6CA20A920629
:103DA200A20B300701B350307D037F04124EEA505C
:103DB2002320070E300B0B9000A8E0FF7C0B7DE068
:103DC200800F30070F200B0C9000A9E0FF7C0C7DC8
:103DD20000125C6CA20B9207A20D300801B35030A6
:103DE2007D047F04124EEA502320080E300D0B9002
:103DF20000AAE0FF7C0C7D20800F30080F200D0C04
:103E02009000ABE0FF7C0C7D40125C6CA20D92082E
:013E1200228D
:1065B500534103900024E0FE543FFF780408800116
:1065C50023D8FD54F0FFEE30E40343070490002484
:0F65D500E030E503430708EF4241C2AF124CD755
:0165E4002294
:022992008F6B49
:10299400302F05756CF48003756C64E56B6401700D
:1029A40029AF417803EF08800123D8FD3392307FAB
:1029B4001020300B122AAE7F10126F8A022AA61240
:1029C4002AB97F10126F9D022AA6E56B6402702853
:1029D400AF417802EF08800123D8FD3392307F2085
:1029E40020300A122AAE7F20126F8A8008122AB978
:1029F4007F20126F9D022AA6E56B64037028AF4105
:102A04007801EF08800123D8FD3392307F402030D5
:102A14000A122AC47F40126F8A8008122ACF7F408C
:102A2400126F9D022AA6E56B6404701EE541339281
:102A3400307F8020300A122AC47F80126F8A800877
:102A4400122ACF7F80126F9D8058E56B6405702732
:102A5400AF417805EF08800123D8FD3392307F041D
:102A640020300A122ADA7F04126F8A8008122AE5BB
:102A74007F04126F9D802BE56B6406702CAF417848
:102A840004EF08800123D8FD3392307F0820300AF8
:102A9400122ADA7F08126F8A8008122AE57F081248
:092AA4006F9DAF6C7E00126CEE18
:102AAD0022126F9DAF6C7E00126CEE22126F8AAFF8
:102ABD006C7E00126CEE22126F9DAF6C7E00126C5C
:102ACD00EE22126F8AAF6C7E00126CEE22126F9D99
:102ADD00AF6C7E00126CEE22126F8AAF6C7E00120C
:032AED006CEE226A
:105DDF00900024E030E0057F10126F9D900024E0CA
:105DEF0030E1057F20126F9D900024E030E2057FA7
:105DFF0040126F9D900024E030E3057F80126F9D6D
:105E0F00900024E030E4057F04126F9D900024E0A1
:095E1F0030E5057F08126F9D2299
:106D3F0030030A124D1BC203C211C21E22300409B6
:0A6D4F00124D1BC204C213C21E2223
:1065E5008F708D71E570B4011FE5717003125D0246
:1065F500E571B40107787FE6FF125B3CE571B432C3
:106605000E7FF47E01026CEEAD71AF7012675822F9
:10675800EFFEEDFF1280008E2D8F2E12546E757491
:1067680032AF741574EFD39400400EE4F573E573FB
:09677800C3943A50EC057380F55E
:0167810022F5
:10546E00D2A8AFA875A881C214852E82852D83E49B
:10547E0093C4540FFE4306F08E80C284D28500C2C0
:10548E00870000D287007580FF7580FEC284C285BA
:10549E0000C2870000D287007580FFD2147D407C49
:1054AE001FE4FE30B40D0EBE32F9ED1D70011CED81
:1054BE004C70EE7C1F7D40E4FE20B40D0EBE32F922
:1054CE00ED1D70011CED4C70EE8FA8C2A87F0A7EF8
:0454DE0000126CEE5E
:0154E20022A7
:106782007580FDC284C28500C28700000000D287E6
:10679200007580FF7F0A7E00126CEE7F997E0912DF
:0A67A20080008E2D8F2E12546E22FF
:10422800D284D285C286A2809217A2819220A282CD
:104238009218A2839221D2862001537D027F011217
:104248004EEA40137D037F01124EEA400A301707F9
:10425800301932D22480377D027F01124EEA500F86
:1042680030170C302009301904D224802180167DA3
:10427800037F01124EEA501220170330200C301928
:1042880004D22480091268268004C219C22420029C
:104298004E7D027F02124EEA40127D037F02124ECB
:1042A800EA4009301806301B2FD225227D027F02F2
:1042B800124EEA500E30180B302108301B03D2255D
:1042C8002280157D037F02124EEA500F201803301A
:1042D8002109301B03D2252202684EC21BC22522A7
:10682600753D1E753E60E4FFE53E2FF582E4353D7D
:10683600F583E4F00FBF50F0753D1E753E60E4F53C
:0768460045C226C211D21960
:01684D002228
:10684E00753F1E7540B0E4FFE5402FF582E4353FFD
:10685E00F583E4F00FBF10F0753F1E7540B0E4F500
:07686E0046C228C213D21B31
:016875002200
:106C7C00C284D285C286A2809209A281920AA28283
:0D6C8C00920BA283920DD286D284D2852273
:1061B000E57D2560F582E4357CF5832274FF123A93
:1061C00034E4FBFAF9F8C3023A21057E7480257D98
:1061D000F57DE4357CF57C22F582E4341DF58322DF
:0B61E000757E01757C00757D20E422B7
:1042E8007D027F07124EEA50057F04126F8AC229A9
:1042F800D223E4F5427FE87E03126CEEC298C2AF87
:10430800C2307F03122ECA755E7F755D96755C9804
:10431800755B00785B1261BC504430983E12000611
:10432800126EA0EF14601824F0602624C1600B24DC
:10433800F670287F06126FAF802112629A801C7F68
:1043480006126FAF126A5A1265B5125E70D22980D2
:104358000A7F06126FAF125AECD2293029B5E478D9
:1043680084F6D2307F01122ECA7F40120016C22F67
:10437800126A147D467F021267587D1E7F071267F6
:10438800587D147F081267587D327F03126758C220
:0D439800307F03122ECA7FFF126F49C2232F
:0143A50022F5
:105AEC001261E0F55F7F02126FAFE57E2402F56173
:105AFC00AF7E126FAFE4F5601261B0E0FF126FAFD2
:105B0C001261B0E02561F5610560E560C3948040E9
:105B1C00E7AF61126FAF7F03126FAF126FB7EF6415
:0F5B2C0015600C1261CA055FE55FC3942240B695
:015B3B002247
:106A5A001261E0F55F1264BC50077F06126FAF80C7
:106A6A00057F15026FAF1261CA055FE55FC3942205
:026A7A0040E3F7
:016A7C0022F7
:1064BC00E4F560126FB774D025601261D8EFF00567
:1064CC0060E560C3948440EB126E7E901E52E0B582
:1064DC000710AE7CAF7DBE0504BF200100126CD24C
:0364EC00D322C3F5
:0164EF00228A
:106CD200E4FF74D22FF582E4341DF583E0FEE57DF6
:0B6CE2002F1261B4EEF0000FBF80E73E
:016CED002284
:106E7E00E4FFFE74D02E1261D8E02FFF0EBE82F317
:016E8E0022E1
:10629A00E4F55FF5657564E0756393756204F5610D
:1062AA0078611261BC50213098F61200068F60E5C1
:1062BA006064046013AF65056574D02F1261D8E578
:0862CA0060F0255FF55F80D84C
:0162D20022A9
:04000600AF99C29854
:01000A0022D3
:086FAF003099FDC2998F99226F
:076FB7003098FDAF99C2986C
:016FBE0022B0
:106D8C000C0102030405060708090A0B0C01020397
:086D9C000405060708090A0BB3
:1067D500AF5FEF3395E0FE75F007EF123A52EE75B5
:1067E500F007A42583F583E0227882E6FF126D7316
:0967F500EF22C295D297D2AF2227
:10691200C22CC2AF126FBF7F83126DA4126B8B1297
:1069220067F77883E66F600B125F3B302B051260CE
:056932003F922CA22C95
:01693700223D
:10603F007983E778866660367883E6FF7886F6EFB1
:10604F007013E552C3940A500C7D077F04124EEA79
:10605F005003125EB57D057F04124EEA5010E541E4
:10606F0054036005123FCAD322123FCAC322C32270
:103FCA00E4F55F900A501267D5700302408E900A9A
:103FDA00511267DC6016788066600302408E900A90
:103FEA00521267D5788766600302408EAF5FEF335F
:103FFA0095E0FE900A531267DCFF787FE6FEEF6ECB
:10400A006020EF601DB4080BEED394014005EE94D6
:10401A0007400FEF6409706CEE64016005EE6407F7
:10402A007062AF5FEF3395E0FE900A541267DCFFCF
:10403A00F46006EF788266704BE55FFD3395E0FC2D
:10404A00900A5575F007ED123A52EC1267E478833C
:10405A00667031D201D20274BD2DF58274003CF52E
:10406A0083E0FFC007EDAE047805C333CE33CED864
:10407A00F92480F582740E3EAD82FCD007125C6C86
:10408A00C201C202055FC3E55F64809493500302D4
:02409A003FCD18
:01409C002201
:105EB5007D087F04124EEA500D7882E6FF126D735D
:105EC500EFC39407402CD2307F01122ECA7F4012B7
:105ED5000016C22F126A14D201D202E4FD7F0A1203
:105EE5004F72C201C2027F50126F49C2307F011248
:035EF5002ECA2290
:105F3B00C2AF126FBF7FBF126DA4126B8B7883A69B
:105F4B0007126B8B7883A607126B8B7882A60712CE
:105F5B006B8B7887A607126B8B7880A607126B8BDF
:105F6B00787FA607126B8B7881A607126FBF12671B
:025F7B00F7220B
:10599000C2AF126FBF7F8E1259DF7F90126DA47F4E
:1059A000A7126DA4126FBF7FBE126DA4E4FF126D2B
:1059B000A47883E6FF126DA47882E6FF126DA478C6
:1059C00087E6FF126DA47880E6FF126DA4787FE66B
:1059D000FF126DA47881E6FF1259DF1267F72212D9
:0B59E0006DA4E4FF126DA4126FBF2243
:105B3C008F72E572B401047D63803EE572B4020697
:105B4C007D087F068035E572B403067D317F0880C1
:105B5C002AE572B404067D617F08801FE572B405E6
:105B6C00067D257F088014E572B406067D597F03F7
:0F5B7C008009E572B407077D487F07126758223A
:026D7300AE0769
:106D7500EE54F0FF780408800103D8FD75F00AA4ED
:066D8500FFEE540F2FFF8A
:016D8B0022E5
:105D02001267EE906D8C93FF1235B878831267F0AC
:105D1200601B78831267F0C3940A50077D327F06B6
:105D22001267587883E6FF126D731235B81267EE68
:105D3200C3940C50067D0A7F0280047D507F0612B8
:0A5D420067587D507F051267582254
:105A43007FF47E01126CEE7D097F06126758788021
:105A5300125A897D0E7F031267587D357F061267C0
:105A6300587D097F061267587887125A897D1E7FF1
:105A7300091267587D1E7F071267587881E6FF1267
:105A83006D731235B822E6FF126D731235B87FF4C9
:065A93007E01126CEE2200
:076FBF00C2B6C295D2952273
:106DA400E4FEC297EF30E002D297C2B6D2B6EFC388
:066DB40013FF0EBE08EC07
:016DBA0022B6
:106B8B00E4FFD297FED2B6C2B6A297E433C4333336
:0F6B9B00335480FDEFC313FFED42070EBE08E633
:016BAA0022C8
:1058D800EF3395E0FE74702FF58274003EF583E097
:1058E800FF22AF5AEF3395E0FEEF222460F5827471
:1058F800013EAD82FCD22922900520E0F547A3E0C5
:10590800F548222450F58274053EAD82FC229000B1
:10591800BAE0FF7C0E7D2022D222D201E4FF22C20F
:0D59280001C2227F1922D222D2307F02223A
:10283100E5527008126F738F5202292CE552B405CC
:10284100081245188F5202292CE552B40B08126D5B
:10285100098F5202292CE552B40A08125D4C8F529D
:1028610002292CE552B40F08125EF88F5202292C6E
:10287100E552B414081223408F5202292CE552B4B8
:102881001908126BE88F5202292CE552B41E081266
:102891006AC38F5202292CE552B42308126B298F87
:1028A1005202292CE552B42807126F578F52807BB0
:1028B100E552B42D0712689E8F52806FE552B432F3
:1028C100071262D38F528063E552B43E07126C0641
:1028D1008F528057E552B43C07126E488F52804B9D
:1028E100E552B43307126B078F52803FE552B44172
:1028F10007126ED18F528033E552B44C07126EE14C
:102901008F528027E552B44407126EF18F52801B1B
:10291100E552B437071257608F52800FE552B43930
:10292100071254E38F528003E4F552E55370061207
:10293100000E8F5322E553B40506126FA68F532262
:10294100E553B40A06126F018F5322E553B40F0603
:10295100126F108F5322E553B41406123B6E8F533E
:1029610022E553B43D06126C248F5322E553B43F44
:10297100061266158F5322E553B443061268768F0B
:102981005322E553B44D06126B4A8F5322E4F5539B
:012991002223
:0D6F730090052AE0F52BA3E0F52C7F052208
:10451800302414201011C21C7D047F01124EEA5071
:10452800037F0B227F0A227F081263B150061245CF
:10453800CE7F0022202408301005C2107F05227D7E
:10454800057F06124EEA501EE5394538701890006E
:10455800B5E0FF7C0D7D80125C6C90052EE0F5388F
:10456800A3E0F53980517D067F06124EEA501EE51C
:104578003C453B70189000B6E0FF7C0D7DA0125CB6
:104588006C900530E0F53BA3E0F53C802A7D077F81
:1045980005124EEA500B300008E52C452B7002C27C
:1045A80000300F08E52C452B7002C20F7884E6B462
:1045B80005057F04125306E551700875510AD22B80
:0645C8001269127F0522BA
:106D0900200F1590053BE0F54E2024037F0522E571
:0B6D19004ED3940050F3D20F7F0A22EB
:105D4C007D077F05124EEA500C7D077F05124EEA47
:105D5C00503230002F7D017F01124EEA5026D23096
:105D6C007F01122ECA7F011200167D027F07124E90
:105D7C00EA50057F04126F9D9000A0E0FF7C0A7D25
:0A5D8C00E0125C6C1259007F0F2238
:105EF80030243DE5484547700C7D087F01124EEA85
:105F080050037F372230030EE53A700A126D3F7F47
:105F18000112001680173026037F14227884E6B415
:105F2800050B7F031253062024037F14227F0F22C0
:035F38007F1422B1
:1023400090053DE0F54B7F01126F49126D3F7D0214
:102350007F07124EEA5009E54B70057F04126F8A21
:102360009000A1E0FF7C0B7D00125C6CD22B126907
:1023700012E545700302246A7C017D001224F250AC
:10238000037F3E227C017D501224D250037F3C22E9
:102390007C017D581224D250037F3C227C017D10A9
:1023A0001224DA50081224E250037F33227C017D8C
:1023B000201224DA500B9000BBE0FF7C0E7D4080A1
:1023C000207C017D281224EA500512591680127CC7
:1023D000017D301224EA50129000B9E0FF7C0E7D9E
:1023E00000125C6C1268267F00227C017D40D2299D
:1023F000E4FF1247E3500C7D067F04124EEA5003BF
:102400007F4C227C017D381224F250037F44227CD1
:10241000017D18C229E4FF1247E3500C7D057F01BE
:10242000124EEA50037F4122E4F55A1258EA78032B
:10243000C333CE33CED8F91258F3E4FF1247E3503A
:102440001BAF5A1258D8C0071258EA7805C333CECA
:1024500033CED8F912590BD007125C21055AC3E5C7
:102460005A648094A840C47F19221224E2500C7D43
:10247000077F05124EEA504B3000487884E670041E
:102480007F0180087884E6B404077F021253068037
:102490002F7884E6B40704760180257D037F061239
:1024A0004EEA501CE557455670169000AFE0FF7C91
:1024B0000C7DC0125C6C900532E0F556A3E0F55738
:1024C0007F19227D077F05124EEA50052000027F0A
:0124D0000506
:1024D10022D229E4FF1247E322D229E4FF1247E383
:1024E100227D077F05124EEA22D229E4FF1247E33B
:0924F10022C229E4FF1247E32294
:106BE8003026031268267D077F05124EEA500620DC
:0E6BF80000037F0522900538E0F54E7F1E2237
:106AC300E54E70037F23227D027F07124EEA5009B1
:106AD300E54B70057F04126F8A3024037F0A227FFF
:026AE3001E2271
:106B29001259007D067F01124EEA500C9000ACE02C
:106B3900FF7C0C7D60125C6C900539E0F54E7F2D71
:016B49002229
:0E6F57007FA0126F49900539E0F54E7F2D2284
:10689E00D22B1269127D027F07124EEA5009E54B88
:1068AE0070057F04126F8AE54E70037F322230240A
:0768BE00037F0A227F2D2257
:1062D300301E037F32227D047F06124EEA501FE5F3
:1062E30055455470199000B0E0FF7C0C7DE0125CC2
:1062F3006C900534E0F554A3E0F5557F3222C230AB
:086303007F01122ECA7F002267
:106E480020220CD222E4FF12055BC2227F00227F9F
:026E58003C22DA
:106C0600202218D2227F40120016D201121D87C2FE
:0E6C1600017F40126F49C2227F19227F3E2269
:106ED10020220A1259201237B3125927227F412248
:106EE10020220A125920126174125927227F44224A
:106EF10020220A12592012562C125927227F44228D
:05000E0000007F052247
:096FA6003025037F0A227F052239
:0F6F01009000A2E0FF7C0B7D20125C6C7F0F22C2
:0F6F10003025093028037F14227F0F227F14229F
:103B6E009000A3E0FF7C0B7D40125C6CE546700379
:103B7E00023C467D017F03124EEA50707C017D08A7
:103B8E00C2297F011247E350037F3F227C017D5003
:103B9E00123C4950037F3D227C017D58123C495016
:103BAE00037F3D227C017D40D2297F011247E350E5
:103BBE000C7D067F04124EEA50037F4D227C017D60
:103BCE0028D2297F011247E35009125916125C6C54
:103BDE007F00227C017D18C2297F011247E3500C21
:103BEE007D057F02124EEA50037F43227D027F0342
:103BFE00124EEA5043E4F55AAF5A1258EC7803C30A
:103C0E0033CE33CED8F91258F37F011247E3501D4D
:103C1E00AF5A1258D8C007AF5A1258EC7805C333B2
:103C2E00CE33CED8F912590BD007125C21055AC3E8
:0A3C3E00E55A648094A840C07F009E
:093C480022D2297F011247E32278
:106C2400202218D222C2307F01122ECA7F01126F95
:0E6C3400497F0112055BC2227F00227F3D22B4
:1066150020222A12592E122ECA7FF47E01126CEE08
:106625007F10120016D202121B86C2027F10126F53
:1066350049C2307F02122ECAC2227F00227F3F222A
:1068760020222212592E122ECA7FF47E01126CEEAD
:10688600D2027F011237B3C202C2307F02122ECA71
:08689600C2227F00227F432291
:106B4A0020221B12592E122ECAD2027F0112617400
:106B5A00C202C2307F02122ECAC2227F00227F4D99
:016B6A002208
:10555300AF5AEF3395E0FE22900520E0F547A3E034
:10556300F54822900522E0F549A3E0F54A2224609C
:10557300F58274013EAD82FCD2292274702FF5822C
:1055830074003EF583E0FF22C202C2227F19222467
:1055930050F58274053EAD82FC22900536E0F5326B
:1055A300A3E0F53322055AC3E55A648094A822D2B6
:0D55B30022C2307F0122D222C2307F0222AC
:10326500E5527006126AE58F5222E552B405061240
:1032750036B78F5222E552B40B061268C58F52221B
:10328500E552B40A061243A68F5222E552B40F0640
:10329500126E5A8F5222E552B4110612581D8F52E2
:1032A50022E552B4120612518A8F5222E552B41405
:1032B50006120A548F5222E552B419061266A48FDB
:1032C5005222E552B41E061266458F5222E552B4CB
:1032D5002306125FBE8F5222E552B42806126F658F
:1032E5008F5222E552B42D061261EB8F5222E55220
:1032F500B4320612630B8F5222E552B43C06126EAD
:103305006C8F5222E552B43D06126D248F5222E590
:1033150052B43E061269A78F5222E552B43F0612F7
:103325006E8F8F5222E552B44106126BAB8F52223B
:10333500E552B44306126A7D8F5222E552B44C061B
:10334500126D598F5222E552B44D06126AA08F5262
:1033550022E552B437061257608F5222E552B4392E
:10336500061254E38F5222E552B4380612672D8FA8
:103375005222E552B43306126B078F5222E552B43E
:0C3385004406126DBB8F5222E4F5522268
:106AE50090052AE0F52BA3E0F52C7D067F02124EDA
:106AF500EA500C90052CE0F529A3E0F52AD21F7F7A
:026B0500052267
:1036B700302414201011C21C7D047F01124EEA50E1
:1036C700037F0B227F0A22302514201211D21C7D82
:1036D700047F02124EEA50037F0B227F0A227F08E3
:1036E7001263B150061245CE7F0022202408301005
:1036F70005C2107F0522202508301205C2127F055A
:10370700227D057F06124EEA501EE53945387018AE
:103717009000B5E0FF7C0D7D80125C6C90052EE07B
:10372700F538A3E0F53980757D067F06124EEA501D
:103737001EE53C453B70189000B6E0FF7C0D7DA070
:10374700125C6C900530E0F53BA3E0F53C804E7DC4
:10375700077F05124EEA500D30000AE52C452B7005
:1037670004C200800B300F08E52C452B7002C20FF6
:103777007D067F02124EEA5019301F16E52A4529A9
:103787007010C21F9000BCE0FF7C0E7D60125C6C65
:10379700800B7884E6B405057F04125306E5517063
:0C37A7000875510AD22B1269127F05220E
:1068C500200F2190053BE0F54E202406201C037F78
:1068D5000522202506301C037F0522E54ED39400B2
:0768E50050E7D20F7F0A22E9
:1043A6007D077F05124EEA50127D077F05124EEA01
:1043B6004003024457200003024457201C3FD230DA
:1043C6007F03122ECA7F0F126F4990000FE0B402CE
:1043D600047F05800990000FE0B403057F011200F9
:1043E6001612555B7D027F07124EEA50057F0412B6
:1043F6006F9D9000A0E0FF7C0A7DE0804E301C514E
:1044060090000FE0FF64026005EF640370437F0FC6
:10441600126F497F051263B1400BD2307F01122E15
:10442600CA7F028009D2307F03122ECA7F0A120089
:10443600167D027F07124EEA50057F04126F9D1209
:1044460055669000A2E0FF7C0B7D20125C6C7F0F0E
:0A4456002212555B1255667F0F22FB
:106E5A00201C063024037F1122301C053025027FB6
:026E6A001222F2
:10581D00302458E5484547700C7D087F01124EEA4B
:10582D0050037F3722300329E53A70257FA0126F90
:10583D004990000FE0B401047F01800990000FE052
:10584D00B402057F05120016E4F542C21EC20380A4
:10585D00173026037F14227884E6B4050B7F0312DC
:0E586D0053062024037F14227F11227F142271
:10518A00301C1030240D20100A7F0A126F49C21CED
:10519A007F0A22301C5230254F20124C3003031252
:1051AA006D3FE54A4549700C7D087F02124EEA5070
:1051BA00037F3822300417E53A70137FA0126F4933
:1051CA007F02120016E4F542C21EC204801730287C
:1051DA00037F14227884E6B4050B7F03125306205A
:1051EA0025037F14227F1222201C1230250F201241
:1051FA000CD21CC2307F02122ECA7F0A227F1422CE
:100A540090053DE0F54B7F0F126F49201C0C900070
:100A6400A1E0FF7C0B7D00125C6C301C0C9000A399
:100A7400E0FF7C0B7D40125C6CE542B403037F1401
:100A840022126D3FE4F5427D027F07124EEA5009BF
:100A9400E54B70057F04126F8AD22B126912301C49
:100AA40003020B97E5457003020B977C017D00124E
:100AB4000D1E50037F3E227C017D50120CEE50032C
:100AC4007F3C227C017D58120CEE50037F3C227C3B
:100AD400017D10120CF65008120D0650037F3322CC
:100AE4007C017D20120CF65003020BFE7C017D2854
:100AF400120D0E500C9000BAE0FF7C0E7D20020C0B
:100B0400077C017D30120D0E500C9000B9E0FF7C83
:100B14000E7D00020C077C017D40D229E4FF1247C0
:100B2400E3500C7D067F04124EEA50037F4C227C76
:100B3400017D38120D1E50037F44227C017D18C2B2
:100B440029E4FF1247E3500C7D057F01124EEA5061
:100B5400037F4122E4F55A125553EF7803C333CE91
:100B640033CED8F9125571E4FF1247E3501D1255E4
:100B74005312557EC007125553EF7805C333CE3355
:100B8400CED8F9125592D007125C211255A840C74D
:100B94007F1922201C03020C8AE5467003020C8A8A
:100BA4007D017F03124EEA4003020C427C017D0862
:100BB400C2297F011247E3500F7F50120016D23032
:100BC4007F02122ECA7F3F227C017D50120CFE5000
:100BD400037F3D227C017D58120CFE50037F3D2291
:100BE4007C017D10120D165008120D0650037F3340
:100BF400227C017D20120D1650129000BBE0FF7C78
:100C04000E7D40125C6C1268267F00227C017D40C0
:100C1400D2297F011247E3500C7D067F04124EEA6D
:100C240050037F4D227C017D18C2297F011247E3C6
:100C3400500C7D057F02124EEA50037F43227D0251
:100C44007F03124EEA503CE4F55A125553EF7803F1
:100C5400C333CE33CED8F91255717F011247E35016
:100C64001D12555312557EC007125553EF7805C314
:100C740033CE33CED8F9125592D007125C211255D7
:100C8400A840C77F1922120D265008120D26504B7A
:100C94003000487884E670047F0180087884E6B4E4
:100CA40004077F02125306802F7884E6B407047683
:100CB4000180257D037F06124EEA501CE5574556F8
:100CC40070169000AFE0FF7C0C7DC0125C6C900548
:100CD40032E0F556A3E0F5577F19227D077F051210
:090CE4004EEA50052000027F05D4
:100CED0022D229E4FF1247E322D229E4FF1247E37F
:100CFD0022D2297F011247E3227D077F05124EEA9A
:100D0D0022D229E4FF1247E322D2297F011247E3C1
:100D1D0022C229E4FF1247E3227D077F05124EEA26
:010D2D0022A3
:1066A400C219C2307F02122ECA3026051268268013
:1066B4000630280312684E7D077F05124EEA500605
:0F66C4002000037F0522900538E0F54E7F1E224F
:10664500E54E70037F23227D027F07124EEA500933
:10665500E54B70057F04126F8A3024062010037FF6
:106665000A22302508201205D21C7F0A227F1E220D
:105FBE00201C0512555B80031255667D067F01126B
:105FCE004EEA5024E5427020201C0B9000ACE0FFFE
:105FDE007C0C7D60800C301C0C9000ADE0FF7C0CC6
:105FEE007D80125C6C7F2822900539E0F54E7F2D66
:015FFE002280
:0E6F65007FA0126F49900539E0F54E7F2D2276
:1061EB00D22B1269127D027F07124EEA5009E54B42
:1061FB0070057F04126F8AE54E601D302406201057
:10620B00037F0A2290000FE064016009302506200D
:0B621B0012037F05227F2D227F32221C
:10630B00301E037F32227D047F06124EEA501FE5BA
:10631B0055455470199000B0E0FF7C0C7DE0125C89
:10632B006C900534E0F554A3E0F5557F3222C23072
:08633B007F01122ECA7F00222F
:106E6C0020220CD222E4FF12055BC2227F00227F7B
:026E7C003C22B6
:1069A70020221FC2307F02122ECAD2227F4012003D
:1069B70016D201121D87C2017F40126F49C2227F82
:0569C70019227F3E22B1
:106E8F0020220BD222D202121B8612558B227F3F59
:016E9F0022D0
:106D24002022151255B2122ECA7F40126F497F01DC
:0B6D340012055BC2227F00227F3D227F
:106BAB002022191255B9122ECA7F10126F49D20129
:0F6BBB00E4FF1237B3C201C2227F19227F4122A9
:106A7D0020221D1255B2122ECA7F40126F49D230FC
:106A8D007F02122ECAD2027F011237B312558B220A
:036A9D007F432212
:106D59002022141255B9122ECAD201E4FF1261740D
:0A6D6900C201C2227F19227F4122DD
:106AA00020221D1255B2122ECA7F40126F49D230D9
:106AB0007F02122ECAD2027F0112617412558B22FC
:036AC0007F4322EF
:106DBB002022111255B9122ECAD202E4FF12562C00
:076DCB0012558B227F4422C8
:10576000D2107D027F07124EEA50057F04126F8A25
:1057700090000FE0FF64016004EFB4030E7F01129C
:105780006F497F401257AF7F01801390000FE0B444
:10579000020F7F05126F497F501257AF7F03126FC0
:1057A0008A7F50126F4930150312559D7F3922129E
:0F57B0000016C22F126A14E4FD7F07124F7222F7
:1054E30030241130150BE53345327005C231126992
:1054F300CC7F3922E47884F6C21090000FE0FF6479
:10550300016005EF64037010D2307F01122ECA7F51
:10551300401255417F01801B90000FE0640270161A
:10552300D2307F03122ECA7F05126F497F50125566
:10553300417F03122ECA7F50126F497F002212004F
:1055430016C22F126A14E4FD7F08124F72C2302272
:10672D00D2127F0A126F497F40120016D22F126AC1
:10673D0014E4FD7F07124F727F03126F8A7F501290
:0B674D006F4930150312559D7F00229C
:106B070030000B9000B8E0FF7C0D7DE0800C20008A
:106B17000E9000B7E0FF7C0D7DC0125C6CB2007F69
:026B2700192231
:106174008F5AE55A24FF922F126A14E55A70127F3F
:1061840040120016D201E4FD7F09124F72C2018051
:1061940015E55AB401107F10120016D202E4FD7FF7
:0C61A40009124F72C2027F50126F492294
:104D4400C201C202D20C7F50126F497F801200163A
:104D540075420390000FE06401701D3024147F013C
:104D6400120016302404E54270F92024057F011254
:104D74006F49E54270E5804C90000FE0FF640260EB
:104D840005EF6403703E30241D7F02126F497F05D6
:104D94001200167F02126F9D302404E54270F92040
:104DA400241E7F0580173025177F02120016202449
:104DB40007302504E54270F62025057F02126F496D
:0E4DC400E54270C27FA0126F49C20CC21E22CF
:03000000026C99F6
:106C9900758E0078FEE4F6D8FD9000007FFF7E1F18
:0D6CA900E4F0A3DFFCDEFA758187024C25C4
:10399800C2D530F707B2D563F0FF05F030E70CB2B7
:1039A800D5F4048463F0FF05F080018430D502F477
:0239B8000422E7
:1039BA00EF8DF0A4A8F0CF8CF0A428CE8DF0A42E21
:0239CA00FE22DB
:1039CC00BC000BBE0029EF8DF084FFADF022E4CCDF
:1039DC00F875F008EF2FFFEE33FEEC33FCEE9DECA8
:1039EC00984005FCEE9DFE0FD5F0E9E4CEFD22EDEE
:1039FC00F8F5F0EE8420D21CFEADF075F008EF2F38
:103A0C00FFED33FD4007985006D5F0F222C398FD28
:053A1C000FD5F0EA22C5
:103A2100EB9FF5F0EA9E42F0E99D42F0E89C45F0FB
:013A31002272
:103A32007401FF3395E0FEFDFC080808E6CF2FF67F
:103A420018E6CE3EF618E6CD3DF618E6CC3CF62258
:0C3A5200A42582F582E5F03583F583227F
:103A5E00D083D082F8E4937012740193700DA3A3F7
:103A6E0093F8740193F5828883E47374029368600B
:063A7E00EFA3A3A380DF0B
:106EA000EFC39461400AEF947B5005EF24E0FF228A
:016EB00022BF
:00000001FF
